:020000020000FC
:0200000037C007
:02000800567828
:100034000C945A2C0C94582C4156522D43686970D8
:100044004261736963322028632920323030362DAF
:1000540032303039204A6F65726720576F6C667290
:04006400616D0000CA
:10007000F894A0E02A2EA1E03A2EA0E1AEBFAFEFA7
:10008000ADBFB0E0A0E0AA95F1F7BA95D9F70E940C
:10009000EE2D0E94393A0E940E790E94D1350E94BD
:1000A000482FAFEFA093310120923D0120923E01F5
:1000B000209250018827789420922D01A091290147
:1000C000A4FD0C946A000E94482F0E94CD010E945A
:1000D000A933CECFA1E00E94BE2EAA270E94682E8F
:1000E0009927A7E10E94B92E0E94482FA0E10E9403
:1000F000B92EC4E0DAE0E7E3F7E10E949132A7E02D
:100100000E94B92E0E94423107042000B5D1A6E119
:100110000E94B92EC5E0D8E0E6E0F9E00E949132F5
:10012000D8E1F9E10E949132D8E0F9E0CC5FEC5FD0
:10013000C833A0F368E70E9480334091140141FD69
:100140000EC06A95C1F756E142E00E947B390E94D9
:1001500080330E9480335A95B9F70C94CC000E94EA
:10016000482F0E94423100004B6579626F617264D2
:100170002D54657374000E94832F70917101A091BA
:100180007101A215E1F32092710190E07A2F0E9493
:10019000332F0E94B32FF3CFA0E00E94BE2EA1E028
:1001A0000E942435992720922A01AA270E94682EAE
:1001B000A5E10E94B92E0E94482FC0E0D0E0EDE1F9
:1001C000F4E10E94E532A1E50E94B92E0E9442317D
:1001D0000101838383838383204156522D436869C1
:1001E000704261736963322082828282828200005F
:1001F000A9E9B4E00AE40D9304EC0D930CE80D9327
:1002000008E20D9302E60D9306EA0D93509606EA76
:100210000D9302E60D9308E20D930CE80D9304ECA8
:100220000D930AE40D9320D240913D014B3008F02C
:10023000442740933D01642F67FD66276B3008F02B
:100240006AE050E06F932BD16F9153955830D1F7FE
:10025000E1D1B6D18BD16F938AD26F91423E11F426
:100260006A95EACF433E11F46395E6CF443E21F40C
:10027000643010F06450E0CF453E21F4673010F454
:100280006C5FDACF6830F8F04A3E11F0443F19F75E
:1002900060933D01683039F44A3EE9F6FBD00E9494
:1002A0005B1CF8D079CF693039F44A3EA1F6F2D020
:1002B0000E942521EFD070CFEDD04A3E61F60E941A
:1002C0002C23E8D069CF4F934091140142FD2AC0FE
:1002D0004F914A3E11F0443F41F460933D01DAD022
:1002E00088270E94CD01D6D057CF413F41F460937B
:1002F0003D01D0D088270E94B701CCD04DCF423FDE
:1003000039F460933D01C6D00E94091EC3D044CF8A
:10031000433F39F460933D01BDD00E946E1EBAD0B8
:100320003BCF99CF4F91413F39F460933D01B2D01B
:100330000E94CD03AFD030CF423F39F460933D01EE
:10034000A9D00E94D023A6D027CF433F39F4609391
:100350003D01A0D00E940B249DD01ECF443F09F741
:1003600060933D0197D00E94150494D015CFA091C1
:100370001601A030E1F70E94890420922D01A0917E
:100380001701A43F09F008CF08D00E94B033A0E0C5
:100390000E94682E0E94482FEACF0E94482F88278B
:1003A000209216010E941C7A3C9645914E3411F41D
:1003B000339609940E94270E20920D01209250013D
:1003C00020922A010E94832FA7E20E94B92E92E078
:1003D000A0913E01A03079F0A33021F4A7E20E9461
:1003E000B92E09C0A0E10E94B92EA0E4A09300019B
:1003F000A0EEA0930101A0913E01A03051F40E9413
:10040000423116002050524553532045534320009B
:100410002EC0A13051F40E94423169002050524553
:10042000535320455343200022C0A23051F40E9470
:10043000423142002050524553532045534320003F
:1004400016C0A33049F40E9442312F00205052457B
:100450005353204553432000A53049F40E944231B4
:100460003800205052455353204553432000A0915B
:100470001601AD3EE1F708950E944231FF41565208
:100480002D436869704261736963322056302E399A
:1004900031000895A0911601A030E1F70895A1E080
:1004A000B3E050FDA95F51FDA25F52FDBA5F4EE27D
:1004B000651709F4429540932C010E945B310E941C
:1004C0004231FF20200040E50E94B42F452F4F5CB1
:1004D0000E94B42F0E944231FF202000B3950E9459
:1004E0005B31452F0E941E7A3C9645914E3481F433
:1004F0000E944231FF2020E6E7202000B3950E94B1
:100500005B310E944231FF2020E8E92020000FC02B
:100510000E944231FF2020D0D1202000B3950E94BC
:100520005B310E944231FF2020D2D3202000452F92
:100530000E941E7AB3950E945B3166E045910E944D
:10054000B42F6A95D9F7B3950E945B3166E0459167
:100550000E94B42F6A95D9F7B3950E945B310E942F
:100560004231FF2020202020200008954AE26A30F6
:1005700009F4429540932C010E9442310F0F202034
:100580002020202000000E944231100F2020D4D5CE
:10059000202000000E944231110F2020D6D72020B9
:1005A00000000E944231120F20494E464F200000A9
:1005B0000E944231130F20202020202000000895A7
:1005C00048E2693009F4429540932C010E9442317F
:1005D0000F0820202020202000000E944231100817
:1005E0002020D8D9202000000E944231110820206C
:1005F000DADB202000000E9442311208434F4E46B1
:10060000494700000E94423113082020202020206A
:10061000000008954CE2683009F4429540932C01A3
:100620000E9442310F0120202020202000000E9443
:10063000423110012020DCDD202000000E944231E8
:1006400011012020DEDF202000000E944231120133
:1006500044464C41534800000E944231130120207F
:100660002020202000000895A0E00E94B92E0E94C2
:100670004231150020202020202020202020202072
:10068000202020202020202020202020202020206A
:1006900020200000A7E20E94B92E0E9442311600DD
:1006A0002020202020200000A0E60E94B92E0E94D9
:1006B000423116062045646974200000A0E40E94BF
:1006C000B92E0E944231160C20536176652000003D
:1006D000A7E10E94B92E0E9442311612204C6F6190
:1006E00064200000AEE6A0932B07A7E30E94B92E7A
:1006F0000E94423116182052756E20000895A0E025
:100700000E94B92EA7E20E94B92E0E944231160023
:100710002020202020200000A0E60E94B92E0E9468
:100720004231160620436F7079200000A0E40E9439
:10073000B92E0E944231160C2053656E64200000D1
:10074000A7E10E94B92E0E94423116122052656321
:1007500076200000AEE6A0932B07A7E30E94B92EF7
:100760000E9442311618436C6561720008953DED98
:10077000209217010E94493440911401447043179C
:1007800039F0342F403011F46FDFF4CFB8DFF2CFFF
:1007900040911701403071F30895A4E00E94B92EF2
:1007A000C1E0DFE0ECE1F3E10E94E532A0E40E9469
:1007B000B92E0E9442311002436F70792050726F3F
:1007C0006772616D20746F0070913D0160E0ACE074
:1007D000671709F4A0E60E94B92EB2E1A62FAA0F6E
:1007E000A60FAD5F0E945B3140E50E94B42F462FFB
:1007F00047704F5C0E94B42F6395683041F70E94A8
:10080000A933423E21F47030D1F37A95DFCF433ED5
:1008100021F47730A1F37395D9CF4A3E19F40E94A1
:10082000517A08954D3E59F708950E942E384F434E
:100830006C65617220746869732050726F677261B1
:100840006D3F2000413009F008950E942B7A0895F1
:10085000AA270E94BE2EA3E00E9424358F934091C8
:100860003D010E9424790E94482F0E945D2E992705
:10087000409116014030E1F70E94423100002050C3
:10088000524F4752414D200040913D014F5C0E9424
:10089000B42F4AE30E94B42FC3EDD1E058D2F0D276
:1008A0000E94EB7903D48F91A8E8803069F1ACEC19
:1008B000E6EEF0E1813031F0ABE48A9545914030CD
:1008C000E9F7F8CF4CD292E0A5E0B1E00E945B31AD
:1008D0000E943A310E944231FF20494E20500000D0
:1008E00040913A014F5C0E94B42F4AE30E94B42F1A
:1008F000BB27AC2DA3950E94D82E4AE30E94B42FAB
:10090000AD2DA3950E94D82E0895AAE25A2E70E22A
:1009100008959927FADF9CDFD22CAA27BB27D09213
:100920002E010E94D3330E944934403E11F4AA277D
:10093000F6CF413E11F4AFE12BC0423E11F4AA952F
:1009400027C0433E69F4A3959B2F0E94AC099A17D8
:1009500030F4BE3511F4AA951BC0AA27B39518C070
:10096000443E21F4BA95B7FDBB2712C0463E21F4A0
:10097000B850B7FDBB270CC0473E11F4B85F08C0A4
:10098000453E11F4B39504C04A3E39F5B395AA2704
:10099000A03838F0AFE1BA95B038C0F0AA27BB272D
:1009A000BECFA03228F0BE3589F0AA27B395B7CFC5
:1009B000BF3508F0BEE50B2F0D1508F4D02E0D2D18
:1009C000015F0B1718F40B2F0F50D02E9B2F0E9496
:1009D000AC099A1708F4A92FA2CF9B2F4E3E39F4E9
:1009E000AF93BF930E946E09BF91AF9189C14F3EF3
:1009F00031F4BF930E947909BF91AA2781C1493E72
:100A000011F482D17DC14C3E31F4A03009F489CF7C
:100A1000AA957AD175C150911401547009F4C5C0DA
:100A2000433FD1F4ACEC9BD10E94423101075245C7
:100A300043454956452050524F4752414D20592F6A
:100A40004E203F006DD12EF48DD230D35EDF509218
:100A5000C8017DD1882761CF423F39F5ACEC7FD109
:100A60000E944231010753454E442050524F475295
:100A7000414D20592F4E203F000052D156F7ACEC8B
:100A80006ED10E944231010753454E44494E472ED4
:100A90002E2E2020202020202020000030922A010D
:100AA00093D120922A0131DFD4CF443FB1F4ACEC92
:100AB00056D10E9442310107434C454152205052C9
:100AC0004F4752414D20592F4E203F0029D126F447
:100AD000DBD21BDF5092C801BCCF413F41F5ACECEB
:100AE0003ED10E94423101075052494E542050528B
:100AF0004F4752414D20592F4E203F0011D1B6F49F
:100B0000ABE42DD10E94423101075052494E544965
:100B10004E472E2E2E202020202020202000A2E034
:100B2000A0932A0151D120922A01EFDE92CF4336C1
:100B300071F462E46093E50165E56093E60166E4C3
:100B40006093E7016DE36093E80179D2EACE48371C
:100B500091F462E46093E50165E56093E60166E483
:100B60006093E7016DE36093E8010E941F087CD267
:100B70005092C80118C04637B1F46091E501623463
:100B800099F460E26093E5016093E6016093E70108
:100B90006093E8016093E9016093EA0143D286D251
:100BA0005092C801BECE8827BCCE423F11F5BF93FC
:100BB000AF93C9D0D9F0ACECD2D00E94423101073A
:100BC000534156452050524F4752414D20592F4EC8
:100BD000203F0000A5D046F40E94B7790E94EB792F
:100BE00065D293DE7093C801B2D08827AF91BF91D0
:100BF00096CE433FE1F4BF93AF93A5D0B9F0ACECF0
:100C0000AED00E94423101074C4F5354204348411B
:100C10004E47455320592F4E203F000081D026F7E4
:100C20000E94EB7943D271DE7093C801DDCF413F62
:100C300049F46A2E7B2EADD0A62DB72D5092C80157
:100C400070CED2CF4D3E09F5BF93AF937CD0A9F0C3
:100C5000ACEC85D00E9442310107515549542057D0
:100C60002F4F205341564520592F4E203F0058D03A
:100C700046F7A0911601A030E1F70E94552EA0E0A2
:100C80000E94682EAF91BF910895443FE1F45BD07C
:100C900029F40E94552E0E94482F0895A9E65FD09E
:100CA0000E944231010753415645204348414E4777
:100CB0004553204245464F52452052554E21000093
:100CC0000E94A93391CF5091140152FD1CC053FDD5
:100CD0001AC04C31C0F04038B0F4AF3171F05A2F27
:100CE000AFE10E9428346A916983AA95A517D9F7C4
:100CF0004883A3955092C80114CE0E94283448839B
:100D00005092C8010ECE0DCE0E9428345A2F5F316A
:100D100021F0498149935395FACF50E258830895C1
:100D20000E94A933493559F0493749F04A3E39F014
:100D30004E3439F04E3629F04D3E19F0F1CF68941B
:100D40000895E8940895A091C801A0320895A8E8F4
:100D500006D00E94423101054F4B00000895EF93E9
:100D6000FF939927A09340010E9442310105202062
:100D70002020202020202020202020202020202073
:100D8000202020202020202020202000FF91EF91F3
:100D90000895A0E00E94FB334A3E09F40895423EC4
:100DA00021F4A030B9F3AA95F5CF433E21F4AB303E
:100DB00089F3A395EFCF403268F3403858F7488362
:100DC000AB3009F0A395E6CFC9ECD1E056E14991EB
:100DD0000E94B42F5A95D9F70E94832F4EE511D067
:100DE00016F04A95E1F7542F53954427451719F00B
:100DF00024D04395FBCF43E20E94B42F0E94832F5F
:100E00000895CF93DF935F936F93E894C4E3D2E0A8
:100E100053E2459FC00DD11D50E26991613238F413
:100E20005A95D9F76F915F91DF91CF9108956894AA
:100E30006F915F91DF91CF910895DF93CF934F939F
:100E40005F936F93C1E3D2E053E2459FC00DD11D84
:100E5000DF93CF93A39653E26A91613210F45A95CF
:100E6000D9F7CF91DF9149910E94B42F5A95D9F7C4
:100E70000E94832F6F915F914F91CF91DF910895E1
:100E8000AF93BF93EF93FF934F93AEE0B2E0E8EAE6
:100E9000FEE04591403011F04D93FBCF4F91FF9113
:100EA000EF91BF91AF91089520457869742020207B
:100EB0004E616D6520202053617665202052656C5F
:100EC0006F616420202052756E202000AF93BF9385
:100ED000EF93FF934F93AEE0B2E0E4EFFEE0459175
:100EE000403011F04D93FBCF4F91FF91EF91BF91A7
:100EF000AF91089520202020202020205072696E7C
:100F000074202053656E6420202052656376202073
:100F100020204E6577202000AF93BF93EF93FF937F
:100F20004F93AEE0B2E0E0E4FFE04591403011F0D5
:100F30004D93FBCF4F91FF91EF91BF91AF910895EA
:100F40002041626F72742020202020202020202049
:100F50002020202020202020202020202020202091
:100F600020202000D9DFACECFADE0E9442310105DE
:100F7000524543454956494E472E2E2E0000209299
:100F80002E010E9444089927ECECE0934001E3ED28
:100F9000F1E0EE2EFF2E41E10E9438355CE00E9428
:100FA00054354B31B9F14A33D1F70E9454354B31A6
:100FB00089F1403218F041935A95B9F7403228F040
:100FC0000E9454354B3131F1F9CFEEE0F2E0EE2ED4
:100FD000FF2E53E2EE2DFF2DB396EE2EFF2E0E9434
:100FE00054354B31B9F04032D0F3433299F006C05A
:100FF0000E9454354B3171F0403248F041935A957C
:10100000B9F70E9454354B3129F04032D0F793950F
:101010009036F9F60895A3E2BA9FA1E3B2E0A00DDD
:10102000B11D0895BF93AF93F6DFC8E7D1E053E257
:1010300049914D935A95E1F7AF91BF910895BF93B0
:10104000AF93E9DFC8E7D1E053E24D9149935A9558
:10105000E1F7409178014093E90140917901409393
:10106000EA01AF91BF910895BF93AF934F935F9300
:10107000D2DF139640E250E24D935A95E9F75F9123
:101080004F91AF91BF910895DF93CF93BF93AF93EB
:101090004F9340E2A1E3B2E0CDEFDCE04D93219726
:1010A000E9F74F91AF91BF91CF91DF91DF93CF934C
:1010B000BF93AF934F9341E0A1E3B2E0C0E3D42FDD
:1010C000DA5010F0C395FCCFD65CCD93DD93C0E22F
:1010D000CD9390964395403689F74F91AF91BF914C
:1010E000CF91DF910895425245414B004F564552F2
:1010F000464C4F5700444956494445202F30005331
:1011000051522046524F4D203C3000434F4E5354D5
:10111000414E5420544F4F204249470057524F4EA2
:10112000472045585052455353494F4E0053594E4E
:10113000544158204552524F5200554E4B4E4F5736
:101140004E204B4559574F52440057524F4E47205F
:10115000464F524D415400424144204C494E454E69
:10116000554D424552004E45585420572F4F20466A
:101170004F520052455455524E20572F4F20474F43
:1011800053554200544F4F204D414E5920474F5325
:10119000554200544F4F204D414E5920464F52006A
:1011A000493243204552524F5200554E4B4E4F57F5
:1011B0004E204552524F520044464C415348204520
:1011C00052524F52004F5554204F462041525241E7
:1011D0005900494E434F4D504C45544520504152C3
:1011E000004B4559574F5244204953204D495353C2
:1011F000494E470057524F4E472042434F505920C7
:10120000004F5554204F462053435245454E00430E
:10121000414E4E4F54204352454154452046494C7F
:1012200045004D454D4F52592046554C4C004649BE
:101230004C45204E4F5420464F554E440050414798
:1012400045204E4F5420494E2046494C45005041C0
:10125000474553204E4F5420494E2052414E47455A
:10126000004E4F5420494E20475241504849435365
:10127000204D4F4445004E4F5420494E2054455870
:1012800054204D4F4445004E4F205553522046495F
:101290004C4500535243204F5554204F4620534352
:1012A0005245454E0044455354204F5554204F4617
:1012B0002053435245454E0057524F4E47205350FE
:1012C0005249544500494F2044495341424C4544FA
:1012D000004E4F204558544D454D0000BE3508F096
:1012E0000895BF9328D0B395BE35E1F7BDDEBF9119
:1012F000DDCEBE3508F00895BF93AF93AB2FAA950E
:10130000BDE508D0BA95BA17E1F7B395ADDEAF9158
:10131000BF91CCCEBF93AF93DF93CF937CDE139678
:10132000ED01B0E2A991AAA3BA95E1F7CF91DF91BF
:10133000AF91BF910895BF93AF93DF93CF936BDECF
:101340001396ED01B0E2ABA1A993BA95E1F7CF9165
:10135000DF91AF91BF910895BF93AF93DF93CF9388
:101360005ADEED0193964E914132E8F34038D8F7BA
:10137000AC1BBC0B9A2F925097FD9927CF91DF9110
:10138000AF91BF910895CAEEDCE02A922A9280E0E4
:101390002F92AA27BB27442771917032E9F37C3141
:1013A00021F4A191BB27719156C07E3121F4A19106
:1013B000BB27719150C07D3121F4B191A191719100
:1013C0004AC07F3121F4B191A191719144C07C3127
:1013D00030F4572F4C2E5D2ECE2FDF2F63C074328A
:1013E000C1F47191703320F07A3310F4705305C05A
:1013F000713468F0773458F47753B03148F4A295DB
:10140000B2955A2F5F70A07FB52BA70FEACF23C0EC
:1014100029C0703350F17A3340F5403810F086E03F
:101420002AC1AA0FBB1FF0F04A2E5B2EAA0FBB1FCA
:10143000C8F0AA0FBB1FB0F0A40DB51D98F07053F3
:10144000A70FB21D78F0B7FD0DC07191703318F081
:101450007A3308F4E6CF4F3709F473D1AA93BA93DD
:1014600040E89DCF85E007C144C07134E8F37B3587
:10147000D8F76081613458F16B3548F54C2E5D2EFC
:10148000CE2FDF2F21970C2F1D2FE2EFFBE152E033
:101490007591703011F488E0EEC0703261F469919A
:1014A000683299F45F93452FAA27BB27EC2FFD2FB5
:1014B000C42DD52D71CF6991671751F37591703295
:1014C000E9F75395C02FD12FE3CF87E0D4C0403840
:1014D00010F086E0D0C07154770FEF93FF93E0E9EE
:1014E000FCE0E70FF21DA191B191FF91EF91719195
:1014F000B2CF7D3251F44F3711F444274DCF20F451
:10150000403210F04FE748CF6FC0783231F471E0CD
:101510007F93AA27BB27472F3FCF793209F05EC0C0
:101520005F91513019F0523011F403D153C0533050
:1015300011F413D14FC0543029F4CCD1803009F0CC
:101540009AC046C0553029F4B991A991B095A0959B
:101550003FC0563009F4DDC1573009F48DC2583010
:1015600009F49EC2593009F4B3C25A3009F4CAC210
:101570005B3009F4D2C25C3009F4D3C25D3009F4A7
:10158000D5C25E3009F4AFC2503109F40AC25131FC
:1015900009F425C1523109F428C1533109F40EC2AE
:1015A000543109F423C25F3009F411C3553109F4F1
:1015B000BCC1563109F4D0C1573109F4D5C15030FE
:1015C00029F06ED0803009F056C0AACF86E0089589
:1015D000AA93BA93AA27BB2742E0DECE4F3720F466
:1015E0004F3010F086E047C07C3361F471E26081D7
:1015F0006E3319F472E2619142C06D3311F473E2FB
:1016000061913DC07E3339F474E260816D3311F431
:1016100075E2619134C07D3311F476E230C07B32E3
:1016200011F470E32CC07D3211F471E328C07332E1
:1016300011F472E324C07A3211F470E420C07F32D6
:1016400011F471E41CC0753211F472E418C07632E2
:1016500011F473E414C05F91503021F05F3130F029
:101660001FD0F9CFB991A9913197089586E05F9184
:101670005030C1F3FCCF4F914030E9F708955F91AE
:10168000A72FB52FA07FB07FBA1720F009D08030E8
:1016900091F7F5CF5F937F93AA27BB27472F7CCE87
:1016A0005F934F9319910991B991A991513211F416
:1016B000FED03AC0523221F4F3D0A150A17034C010
:1016C000533221F4FCD0A150A1702EC0543211F439
:1016D000F6D02AC0553221F4EAD0A150A17024C01E
:1016E000563211F4DDD020C0503311F441D01CC06B
:1016F000513311F43CD018C0523319F4A02BB12B44
:1017000013C0503411F43FD00FC0513411F4A7D09E
:101710000BC0523421F4A3D0A22FB32F05C05334F1
:1017200019F4A023B12300C0AA93BA934F915F91FB
:101730000895B991A99103D0AA93BA930895B7FFD8
:101740000895A095B095A30DB21D089517FF0895B3
:1017500000951095030D121D0895B991A991AB2B19
:1017600029F0B7FBA1E0BB270EF41297E5CFF0DF1D
:101770002B2F2127A00FB11F27FD08952B2F2127E5
:1017800027FD82E008950CD0A22FB32FBF770EF46F
:10179000D8DF37FD03C0452B09F4089582E0089592
:1017A0007AD0CDDFB19F402D512DA09F202D312D1E
:1017B000A19F300D411D521DB09F300D411D521D86
:1017C000089508E611E0B03818F0A00FB11FFBCF64
:1017D000A017B10718F0A01BB10BFACF0895B9916B
:1017E000A9910AE5A01BB20902C0B991A991E9DF4C
:1017F000FF93EF93E2E9FCE70AE510E0A017B107D9
:1018000048F4E00FF11FEA1BFB0BA491EF91FF914D
:10181000BB27DECE04EB10E0A017B10778F40AE591
:1018200010E0E01BF10BEA0FFB1FA491EF91FF9179
:10183000BB27A095B095A30DB21DCACE0EE011E056
:10184000A017B10728F4E00FF11FEA1BFB0BEDCF47
:101850000EE011E0E01BF10BEA0FFB1FD6CF212FAA
:10186000202B11F483E0089516D022273327442734
:1018700051E1441FAA1FBB1F5A9551F0221F331F6D
:101880004FEF201B310BA8F7200F311F40E0F1CFA5
:101890000EF457CF08952B2F212727FB50DF56CF6B
:1018A0000A271B27AA27BB27012B89F00895B058C8
:1018B0001058A01BB10BAA27BB2748F00895B058B9
:1018C00010580A1B1B0BAA27BB2708F00895A1E09C
:1018D000B0E00895B991A99184E0B7FD08950F9300
:1018E0001F932F933F9388270A2F1B2FB2E0AA271D
:1018F000232D3327021B130B20F0A3952B0F321D32
:10190000F9CFBB27AA93BA933F912F911F910F91C3
:1019100008954F935F930E94E0351991099142DF3A
:10192000A42FB52F5F914F9153CE19910991023099
:1019300039F420925001A2E0A0933301BB2748CE96
:10194000013031F4A0913301A03011F43092330111
:10195000A0913301BB273CCE199109910EBD0E9485
:101960002B18AEB5BB2734CE10913E01103011F0CC
:101970008CE1089519910991A4ECB2E00A171B07B4
:1019800010F082E10895FF93EF93FDE0ECE3E00FA8
:10199000F11F68940E946B35EF91FF91A42FBB2734
:1019A00017CEB991B0937301A991A0937201CF930F
:1019B000DF930E942F18DF91CF910ACEB991A991A0
:1019C000BF3F71F0A09358010E940521803021F0A3
:1019D000AFEFBFEF8827FCCDA42FBB270C94E80AFC
:1019E0000E940A218827B42FAA27F2CDB991A99184
:1019F000BF3F21F5A0FD11C0DF93CF93FF93EF937D
:101A00000E940221803019F08827CC27DD27DE01D3
:101A1000EF91FF91CF91DF91DBCDDF93CF93FF93D8
:101A2000EF930E940221803019F08827EE27FF27CC
:101A3000DF01EF91FF91CF91DF91CACDA0935801C3
:101A40000E940521803021F08827AA27BB27C0CD1E
:101A5000DF93CF937F9377270E940D21DF3F41F4DF
:101A6000CF3F31F4A72FBB277F91CF91DF91B0CD2E
:101A70007395703889F7F6CFA991A991A770A06CDA
:101A8000A0937C00A0917A00A064A0937A00A0911A
:101A90007A00A6FDFCCFA0917800B091790098CD96
:101AA000B991A991B03061F4AF3F79F0A770A395D7
:101AB000B0B1B695AA95E9F7AA27AA1FBB2788CD8A
:101AC000BA2FA0B1AB23BB2783CDA0B1BB2780CD5C
:101AD000B991A9910E941A790E94763A8030C9F48E
:101AE000BB27A52F75CDB991A991CF93DF93CA2FAD
:101AF000DB2F0E94B63ADF91CF91803051F4BB27A3
:101B0000A42F66CDA99179910E94943A803009F46E
:101B10005FCDAA27BB278FE0AACDB991A991BB279A
:101B200057CDB991A991AB2FBB2752CD0F93B99146
:101B30000991AA27BB27003019F4A091160145C0CE
:101B4000013029F4A0911601A030E1F33EC002302B
:101B500039F4A0911601A030E1F7A091170135C02A
:101B6000033019F4A091140130C0043039F400910D
:101B7000140100FD119602FD119727C0053039F4BC
:101B80000091140101FD119603FD11971EC006304E
:101B900049F400911601023E09F41197033EA9F49D
:101BA000119613C0073049F400911601043E09F460
:101BB0001196053E51F4119708C01F93109116011C
:101BC0000117E1F71F91A02FBB270F9101CDB9910C
:101BD000A991BB27A13021F4A0916D01A395F8CC68
:101BE000A23021F4A0916E01A395F2CCA0916F01D7
:101BF000EFCC4142532053474E20535152204E4F79
:101C00005420524E442041444320494E20585045D0
:101C1000454B2054454D50204C4F204849204B45C2
:101C20005920455045454B204552522041522053A2
:101C3000494E20434F53204654595045204653495E
:101C40005A45205053544154205350492000FCE041
:101C5000E0E9A0E0B4EBA193BA95E9F7F1E0E8E69A
:101C6000B0E1A193BA95E9F7FDE0ECE3B0E0A19310
:101C7000A193A193BA95D9F7DD24CC2420920F012A
:101C800020920D01AEE0A0932C01ACE3A09344019F
:101C9000AEE2A0934501AFEFA09377010E94482FD9
:101CA00020925001A2E0A0933301A6ECA0937A0009
:101CB00040913D0140933A01409337010E942479BD
:101CC0009C2D0E94407921D0803039F4AC2DAF3565
:101CD000B8F39CE0209250010895C0926D01D0921B
:101CE0006E0180936F01813051F02092500140913C
:101CF00077014F3520F4DD24C42E8827E1CF9CE006
:101D0000209250010895F70129C0F1E0E0EA209205
:101D10002A018827AD2DBB27AB1701F171917F3FB9
:101D2000F1F17C31C9F07E31B9F07D31A1F07F3124
:101D300091F07732A1F1723241F471917F3F79F1E4
:101D4000773269F17232C9F7E9CF7A3339F7B3954F
:101D5000AB1721F703C071917191E0CF70912D0104
:101D600070FF05C081E07E7F70932D01089572FFA2
:101D700011C0AB7F70932D01A0913E01A53011F0F1
:101D8000A03011F40E945F1BA0FF04C00F900F90C1
:101D900081E008950E94493471917F3F19F4DD2458
:101DA000C394089577FD2BC07032C1F27A3311F4D9
:101DB000D394D4CF773299F37134D8F07B3528F0AF
:101DC00070527134B0F07B35A0F4672E0E94671713
:101DD0007D3379F4D8DA803069F4762D7154770F39
:101DE000DCE0C0E9C70FD21DA993B9938DCFEF9165
:101DF000FF9187E00895703810F487E084CF7F0169
:101E0000E6E0FFE07F73E70FF21D099445C0EFC0E5
:101E1000A2C238C10EC1EFC230C33AC738C339C3FA
:101E20003DC334C088C6A6C64EC3A4C3D6C2FCC335
:101E30002CC47AC16EC47EC483C4EBC197C288C46B
:101E400093C49AC452C54CC1D7C079C22DC1DAC45B
:101E50009DC41CC0DBC4FCC450C2DFC2BFC5A6C742
:101E600011C61DC622C675C1A4C6F5C677C723C64E
:101E700032C65CC20DC554C621C183C299C302C318
:101E800095C497C43FC177C136C694C188E0089510
:101E900084E1089583E108950E946B179CE0732C00
:101EA00020922A01B191B032E9F3BA3321F0B7326E
:101EB00011F0BF3F59F4319770FC0E94832F40917D
:101EC0002A01443010F00E94403A1ECFBB3311F477
:101ED0007724E8CFBC3291F440912A01403031F4AC
:101EE0000E94B32FBA2DB770D9F706C00E94B32F46
:101EF000B0912B01B770D1F77724D4CF732CB332C4
:101F0000C9F420925801209259013DDA4A2F40939A
:101F10002A01443018F4433001F4C4CF0E94443AFB
:101F2000683051F550912A015E7F0E94463A68312F
:101F300019F5B8CFB03411F59AD740912A01433042
:101F400018F40E945B31AECF39F4A0935801B093DE
:101F50005901A0932B01A6CF5FEF0E94463A683249
:101F600059F45A2F0E94463A683231F45B2F0E948E
:101F7000463A683209F496CF8FE00895B13229F4D9
:101F800002DA9A2F8FCF97CF8DCFB23241F44191A1
:101F90004F3FC9F34232C1F30E94B42FF8CFB6329B
:101FA00091F4F1D9B33010F082E10895CCE3DDE093
:101FB000CA0FDB1F4991403029F00E94B42F1196BF
:101FC000B330C0F36FCFB53229F4DDD94A2F0E9468
:101FD000B42F68CF3197D7D9803009F00895903861
:101FE00018F40E94D82E5ECF0E94332F5BCFA0E062
:101FF000F0D60E94482F87CEA2E0EBD6A030C1F0E9
:10200000A13059F0A0915A01A770AA0FB0912C01EC
:10201000B770A295BA2BB0932C01A0915801A7706C
:10202000AA0FB0912C01B07FBA2BB0932C016BCECC
:1020300031CFA3E0CED6A33018F1A0915801B091D2
:102040005901A0937201B0937301A0915A01B0910C
:102050005B01A0935801B0935901A0915C01B0912C
:102060005D01B03011F4A03051F00D010E942F1825
:102070000E94C017D001803021F41197F2CF43CED7
:1020800009CF0895A5E0A5D6A43068F0B0D77F9316
:10209000DDD6E0936B01F0936C010E946F327F916B
:1020A00070932C0130CEF6CEA1E093D6A130D8F3B8
:1020B00040915801417040930D0125CEA5E089D68D
:1020C000A43068F094D77F93C1D6E0936B01F0936E
:1020D0006C010E9491327F9170932C0114CEDACE64
:1020E000A5E077D6A43068F082D77F93AFD6C093AF
:1020F0006B01D0936C010E947B377F9170932C0110
:1021000002CEC8CEA5E065D6A43068F070D77F9324
:102110009DD6C0936B01D0936C010E94CB377F9109
:1021200070932C01F0CDB6CEA3E053D6A23080F050
:102130005ED77F93B0915801A0915A01A0936B0193
:10214000B0936C010E946E317F9170932C01DBCDB6
:10215000A1CEA5E03ED6A43068F049D77F9376D6CD
:10216000E0936B01F0936C010E944B337F9170936D
:102170002C01C9CD8FCEA0913E01A03011F08CE191
:102180000895A1E026D6A130A8F3A0915801B091FE
:102190005901CCE3DDE0CA0FDB1F40912C014F93C6
:1021A000AF92BF920E941238BF90AF904F91409370
:1021B0002C01A9CDA0913E01A03011F08CE1089531
:1021C0006FD6C0937201D093730181D67C32F9F43B
:1021D000A1E000D6A13070F2A0915801B091590150
:1021E000CCE3DDE0CA0FDB1F40912C014F93AF928F
:1021F000BF920E943B38BF90AF90C0917201D091C6
:102200007301499329924F9140932C017CCD87E033
:102210007ACDA0913E01A03011F08CE1089540D616
:10222000C0937201D093730152D67C3281F7A1E042
:10223000D1D5A13009F02ECEFF93EF93AF92BF928C
:1022400040912C014F937F934F7040932C010E943B
:10225000F419C1E0D2E0ECE1F5E10E94E532C09171
:102260002C01C295C0932C010E9442310302000050
:10227000A0915801B0915901CCE3DDE0CA0FDB1FFA
:10228000A6E14991403230F0403820F40E94B42F4A
:10229000AA95B9F7772761E025D00E941A1A623013
:1022A00079F4C0917201D0917301799329927F9151
:1022B0004F9140932C01BF90AF90EF91FF9123CDB0
:1022C0007F914F9140932C01BF90AF90EF91FF9180
:1022D000C0917201D09173014FEF4993499313CD8F
:1022E00087E011CD0E940B188827603009F408950B
:1022F0000E94AD1E882762E00895A3E06AD5A2304F
:10230000A0F075D67F93D0916C01C0916B01F091D4
:102310005801E0915A01E0936B01F0936C010E9427
:102320004B337F9170932C01EECCB4CDA4E051D50A
:10233000A43021F48BD50E944732E5CCABCDA1E08F
:1023400048D5A13090F0A0915801A295AA0FAF7E78
:10235000A0930F01D8CCA1E03CD5A13030F0A091E2
:102360005801A150CA2EDD24089594CDA1E031D5A5
:10237000A130D8F3A0915801A150A0937701C3CC0C
:1023800089CDA5E026D5A23030F1F1E0E0915801E9
:10239000E770B0915A01B770BB0FB295B193A230FC
:1023A000C9F0E770B0915C01B770BB0FB295B19303
:1023B000A33081F0E770B0915E01B770BB0FB295AA
:1023C000B193A43039F0E770B0916001B770BB0FE2
:1023D000B295B19398CC5ECD5DCDA1E0FAD4A13099
:1023E000D8F3A0915801A53009F0A3700E94682E7F
:1023F0000E94482F88CCA1E0ECD4A13068F0A091D5
:102400005801B0915901B03019F4A03009F47BCCD7
:102410000E9480331197F7CF3DCD20925001A2E06A
:10242000A0933301A3E0D5D4A33020F1CCE3DDE0C9
:10243000A0915801B0915901B330E8F4AC0FBD1F21
:10244000A0935201A0935401B0935301B09355014E
:10245000A0915A01B0915B01B33068F4AC0FBD1F7D
:10246000A0935601B0935701A0915C01A093500135
:102470002092330148CC82E146CC20925001BF919A
:10248000BF9108952AD5AB2B09F489CC3DCC23D537
:102490003BCCF701ECD40E945B3136CC1ED50E94B8
:1024A000893332CC672F6F9318D56F914A2F0E94D2
:1024B000B42F65FD0E9431340BD57C3271F707D5FE
:1024C0000E94C309F3CFA2E084D4A13019F0A23056
:1024D00021F1E0CCA0915801AA95AF3510F08AE027
:1024E00012CCB0917001BF3010F08DE00CCCAF93E6
:1024F000CCEEDCE0A5E0AB9FC00DD11DB395B09351
:102500007001BD2DB395B068B993BC2DB993B0914E
:102510003D01B993DD24CF900895A0915A01AA9569
:10252000AF35E8F6B0915801BA95B770B09337015E
:10253000B0917001BF3010F08DE0E5CBAF93CCEEE1
:10254000DCE0A5E0AB9FC00DD11DB395B093700149
:10255000BD2DB395B068B993BC2DB993B0913A0134
:10256000B993DD24CF904091370140933A010E9406
:1025700024790895B0D4B0917001B03011F48CE09A
:102580000895BA95CCEEDCE0A5E0AB9FC00DD11D5F
:10259000B0937001B991B7FFF2CFBF77DB2EC9902E
:1025A000499140933A010E942479089587E0089563
:1025B00092D48DD47134D0F37B35C0F77154770F3A
:1025C000672E85D47D3391F70E94C309803009F0CE
:1025D0000895DCE0C0E9C60DD21DA993B99377D464
:1025E000743521F771917F3409F70E94C3094A2E8F
:1025F0005B2E803009F00895B0917001BF3010F06B
:102600008EE00895CCEEDCE0A5E0AB9FC00DD11DBF
:10261000B395B0937001BD2DB395B993BC2DB9930B
:1026200069924992599270CB56D4B0917001B030F2
:1026300011F48BE00895BA95CCEEDCE0A5E0AB9FF9
:10264000C00DD11DB991B7FDF4CFBF77B0936A012A
:1026500059907991BCE0A0E9A70FB21D0D911D9191
:10266000030D121D1E930E93A991B99111960A178D
:1026700041F41B1731F4B0917001BA95B093700119
:1026800043CBC52CD0906A010895A0913E01A030A3
:1026900011F08CE108951FD4BFEFB0937801B19190
:1026A000B032E9F34B2FBF3F21F40E94832F3197C3
:1026B0002BCBBA33D1F3BB3391F3BC3231F40E944C
:1026C000B32FBA2DB770D9F7EACFB23241F44191A6
:1026D0004F3F59F3423219F30E94B42FF8CFB1346F
:1026E000B0F0BB35A0F4B154BB0FB0936A01B08118
:1026F000B13418F0BB3508F40AC0F2D3DCE0C0E90D
:1027000010916A01C10FD21DA993B993C8CF87E078
:102710000895E3D3803009F0F7CA4A2F4B2BE1F339
:10272000409122014030E1F3409122014030E1F735
:102730001197F3CFD2D3A0932301B0932401EDCF0F
:10274000AFD3A0912301A993A0912401A993DCCA3E
:10275000C4D34A2F0E943835BBD37C3221F4B7D37F
:102760000E94C309F6CFD0CA0E944435A42FBB27CC
:1027700097D3A993B993C8CAF70185D34A2FD73005
:1027800020F4C03D10F40E94BF3ABECAF7017BD3CB
:102790005A2FAC2FBD2F0E941A790E94893A0E94AD
:1027A00080330E9480330E948033AECA96D3A1B991
:1027B000ABCAF70168D3D030B1F4BC2FB770B39572
:1027C00077276FE7A0FD70E8A0FD6FEF77FB770F2D
:1027D00070F967FB660F60F9BA95C1F702B1072B74
:1027E000062302B991CAD13041F4B2B1C095BC23DD
:1027F000C095CA23BC2BB2B987CAD230E9F70E9470
:10280000191882CA6AD30E9424357ECA49D3C0935C
:102810007201D093730109911991105858D37C32E9
:10282000A9F431D3B058D058C017D10710F00C2FED
:102830001D2FA017B10710F40A2F1B2FD091730181
:10284000C09172011058099319935ECA86E00895E9
:10285000A0913E01A03011F08CE1089521D3C093E6
:102860007201D093730133D37C3281F700D3C8EC6B
:10287000D1E07EE17B9FC00DD11DCA0FD21DBB27C9
:10288000A881D0917301C0917201A993B9933CCAF8
:10289000A0913E01A03011F08CE1089501D3C093C6
:1028A0007201D093730113D37C3281F6E0D2C8EC6D
:1028B000D1E07EE17B9FC00DD11DCA0FD21DA2EBDE
:1028C000CA0FA2E0DA0FBB27A881A695BA2FA77777
:1028D000B295B078AB2BBB27D0917301C091720138
:1028E000A993B99311CA86E00895DAD2C093720110
:1028F000D0937301ECD27C32B1F7B9D2C8ECD1E0FD
:1029000070913E017770703021F5AF93BF93A6951B
:10291000B6957EE17B9FC00DD11DCA0FD21D788177
:10292000BF91AF91A0FD7695B0FD7695B0FD7695FF
:10293000A2EBB2E0CA0FDB1FA88170FFA295A6959B
:10294000A770BB27D0917301C0917201A993B9936D
:10295000DBC97130B9F4AF93A695A695A69575E13C
:102960007B9FC00DD11DCA0FD21D7881AF91A2FDF2
:102970007295A1FD7695A1FD7695A0FD7695717075
:10298000A72FDECF7230A1F4AF93A695A6957EE176
:102990007B9FC00DD11DCA0FD21D7881AF91A1FDC3
:1029A0007295A0FD7695A0FD76957370A72FC8CF80
:1029B000733071F4AF93A6957AE27B9FC00DD11D61
:1029C000CA0FD21D7881AF91A0FF7295A72FB8CF03
:1029D000AF93A695A695A69570E1C2CFA0913E01B2
:1029E000A03011F08CE10895A3E0F3D1A33080F082
:1029F000A0915801B0915901B33010F082E10895CF
:102A0000B23039F4A73F28F082E1089581E20895B9
:102A100041CACCE3DDE0CA0FDB1FC0934601D0936F
:102A20004901AC81A03091F3AE3180F7BB81B03069
:102A300069F3B73158F7C0915801D09159012596E3
:102A4000BA9F000C111C000C111CC00DC11DD3300D
:102A5000E8F6D0915A01C0915C01C0934801D0932F
:102A60004B01CF3F51F0DF3F41F0CA0FCA95CE3145
:102A700038F4DB0FDA95D73118F40E94AD3843C92A
:102A800086E10895A0913E01A03011F08CE10895F7
:102A900022D2A0912D01A460A0932D0135C9A0914F
:102AA0002901A062A09329012FC9A0912901AF7D1E
:102AB000A093290129C9A3E08CD1A33009F0EAC968
:102AC0000E940521403310F08EE108950E941921E3
:102AD0008030D9F718C9A3E07CD1A33009F0DAC956
:102AE0000E940521403310F08EE108950E941C21C0
:102AF0008030D9F708C9A3E06CD1A23019F0A33017
:102B000021F0C8C9A4E1A0935C010E941321803088
:102B100009F4F9C808950E941621803059F4F3C8C9
:102B2000A1E057D1A13009F0B5C90E940521443177
:102B300091F38EE10895A2E04CD1A23009F0AAC928
:102B4000A0915801B091590140915A01CCE3DDE0C8
:102B5000403041F0D395413029F0D395423011F007
:102B600082E108950E94273B0E94163C803009F0C4
:102B70000895C9C8A2E02DD1A23009F08BC9A09157
:102B80005801B091590140915A01CCE3DDE0403049
:102B900041F0D395413029F0D395423011F082E1D4
:102BA00008950E94E03B0E94433B803011F308955A
:102BB0004EC0F70140D1A09374010E94443A68309E
:102BC000B9F790FF28C0592F0E94463A603481F728
:102BD000A030C9F0DDE0CCE3409174014B0F4A1BFB
:102BE000C40FD21DA13039F00E944A3A603579F500
:102BF0005883AA95EFCF0E944F3A683541F5588324
:102C00000E94403A81C80E944A3A5030A1F3509342
:102C10007401A52FDFCF592F0E94463A6831B9F4CD
:102C20003A2FDDE0CCE3409174014B0F4A1BC40FF7
:102C3000D21D5881503011F4303031F00E94463AA4
:102C4000683229F4AA9569F70E94403A5DC88FE07E
:102C50000E94403A089541D1A0935801B093590180
:102C600037D17C3249F4319632D1723231F031971A
:102C70000E94C30985D1F4CF47C87191723231F0F7
:102C80007F3F21F0BB27A72F7BD1F7CF7081E8CF03
:102C9000A0913E01A03011F48DE10895A7E099D0F4
:102CA000B0915801B0934C01B13039F0B23009F114
:102CB000B33009F43CC085E10895A730E1F7C8E5D9
:102CC000D1E0BA81B0934901BC81B0934601BE8185
:102CD000B0934A01B885B0934701BA85B0934B01D0
:102CE000BC85B09348010E940536803009F00895F4
:102CF0000AC8A63001F7C8E5D1E0BA81B09349010E
:102D0000BC81B0934601BE81B0934A01B885B093AF
:102D10004701BA85B0934801BB85B0934B010E942F
:102D20000536803009F008950C94830EC4CFA4308A
:102D3000E9F7C8E5D1E0BA81B0934601BB81B09311
:102D40004901BC81B0934B01BE81B09348010E9400
:102D50000536803009F008950C94830EA0913E0151
:102D6000A03011F08CE10895F7018DD0C093580187
:102D7000D093590150917401A51708F45A2FA8E770
:102D8000B1E0503071F04D91A0937501B093760190
:102D9000A42FBB27F5D0A0917501B09176015A956B
:102DA000F0CFAA27BB27ECD00C94840EA0913E0153
:102DB000A03011F08CE10895A1E00BD0A13040F0DB
:102DC000A09158014A2F43700E947B390C94830EC6
:102DD00061C8F701A03009F40895DF93CF93C8E5E7
:102DE000D1E040E05A2F503029F4A42F7F01CF9139
:102DF000DF910895DF93CF934F935F930E94C309B0
:102E00005F914F91CF91DF91893121F488277F0124
:102E1000A42F0895A993B99343955A95503019F367
:102E200071917032E9F37C3229F33197A42F7F013D
:102E3000CF91DF910895A3E0CCDFA33009F5909105
:102E40005801B0915A01A0915C010895D0915801A8
:102E5000C0915A01F0915C01E0915E01C09346017E
:102E6000D0934901E0934701F0934A010895A2E00D
:102E7000B1DFA23029F4B0915801A0915A01089510
:102E8000AF91AF9107C8A2E0A5DFA230C9F7C0910A
:102E90005801D0915901A0915A01B0915B01089558
:102EA000F70115D0713478F07B3538F47154770F11
:102EB000DCE0C0E9C70FD21D0895713620F07B37E2
:102EC00010F47156F4CF8F918F9187E0089571912E
:102ED0007032E9F30895F7010895F7010C94C309DE
:102EE000EF93FF930E941534EC2FFD2F00E00E941A
:102EF000B53370912D01713011F4872F08C04A3E0F
:102F0000C9F400937401003031F4AA27BB27882745
:102F1000FF91EF910895C8E7D1E0A191A9930A9597
:102F2000E1F7A0E2A993AFEFA993E8E7F1E00E94EF
:102F3000C309EDCF4C3E49F40030C9F2AA940E9477
:102F40001534A0E2A8830A95D2CF403248F24B371D
:102F500038F6AA2DAD3120F60E94B42F0395C7CFC5
:102F600092E0BB27AC2DA3950E94D82E4AE30E9485
:102F7000B42FBB27AD2D0E94D82E0E94B32F0895E9
:102F8000DF93CF93BF93AF93A0915801B0915901B4
:102F9000B33098F4CCE3DDE0CA0FDB1FAF91BF91F3
:102FA000A883C0915801D09159012196C09358012E
:102FB000D0935901CF91DF910895B45090F0AA0FAA
:102FC000BB1FB33070F4CCE3DDE0CA0FDB1FAF9161
:102FD000BF91A993B993C0915801D09159012296FC
:102FE000E5CF82E1AF91BF91CF91DF9108957091CC
:102FF0002C01A0FF0895A33059F450915C015F703B
:10300000550F707F572B70912C0150932C01089510
:1030100050916001F4CF0E941F21403011F46627C7
:103020000895409360010E941021413009F0662705
:103030000895AF3F31F42C9A2CBCACE5ACBD3DBC3F
:103040000895A7F92CBCAF73A064ACBD3DBCA5B17D
:10305000A4FBA5B90895BDB5B7FFFDCF0895509164
:10306000720140917301433038F4DDE0CCE3C50FC9
:10307000D41FA991BB2710C05050444058F0550FA1
:10308000441F433038F4DDE0CCE3C50FD41FA991D1
:10309000B99102C082E1089540917201509173018B
:1030A000430D521D4093720150937301803009F417
:1030B00008954F914F910895A0EAB1E04FEF52E289
:1030C0004D935A95E9F7C8E9D1E040E25A91503260
:1030D00011F44A95D9F7442EA0EAB1E0C8E7D1E04F
:1030E0004C0EA03C28F4C41518F44881403009F473
:1030F000089593D04F3FE1F37AD04F3FC9F340306A
:1031000081F798D0403069F73DD0403051F70AD070
:10311000403039F74991413618F04B3708F44052A6
:103120004D93DFCF4881403320F04A3310F44053B1
:1031300002C044270895642F7727219648814033A1
:1031400080F04A3370F44053660F771F0B01660F0F
:10315000771F660F771F600D711D640F721D21961A
:10316000EDCF703029F04DE14D937D936D9308952F
:103170006A3020F04CE14D936D930895605D6D933E
:103180004CE108954881443211F0442708956627A0
:103190007727219658815033F8F05A3310F4505362
:1031A0000BC05134C8F0573410F4575305C0513692
:1031B00098F0573688F457555F705295550F661F33
:1031C000771F550F661F771F550F661F771F550F07
:1031D000661F771F2196DECF703029F04FE14D93A7
:1031E0007D936D9308954EE14D936D9308954881BD
:1031F000423211F04427089521964D93499142326D
:1032000019F44D9341E00895403029F442E24D9382
:103210004FEF4D9308954D93F1CF4881473211F010
:103220004427089521964D9349914030E1F74FEF9F
:103230004D930895FF93EF93BF93AF935F93EEE4A5
:10324000F9E40E014591403089F0689457E0A5916A
:10325000AE3239F0B991B13608F0B052AB1709F07F
:10326000E8945A95A1F716F0E001EBCF5F91AF918A
:10327000BF91EF91FF91403041F04D934F934881C2
:10328000403211F42196FBCF4F910895CBE7D1E066
:10329000A0EAB1E040E2E0E24993EA95E9F7A097BD
:1032A000A03C29F04D91423010F04F3F11F429928B
:1032B0000895403220F0403810F486D0F1CF4C31E0
:1032C00021F4ED91FF2719D0EBCF4D3121F4FD9181
:1032D000ED9113D0E5CF4E3131F444E275D0ED914C
:1032E000FF273CD0DDCF4F3131F444E26DD0FD916A
:1032F000ED9134D0D5CF50D0D3CFE8944FE2439561
:10330000E051F742E0F7E05FF84D403311F063D051
:1033100068944FE24395E85EF340E0F7E851FC4FD4
:1033200016F0403311F057D068944FE24395E456BD
:10333000F040E0F7EC59FF4F16F0403311F04BD05E
:1033400068944FE24395EA50E8F7E65F16F04033A1
:1033500009F041D040E34E0F3ED00895E8944F2F3E
:1033600042954F7011F012D068944F2F4F700EF0AD
:1033700011F00CD068944E2F42954F700EF011F062
:1033800005D068944E2F4F7001D00895405D4A33A8
:1033900008F0495F20D00895EEE4F9E455915030EB
:1033A00009F40895451711F03796F8CF5F9357E069
:1033B00045914E3209F00FD05A95D1F75F915C31AB
:1033C00010F040E208D008954993CB3918F02992C3
:1033D0004F914F9108954993CB3928F029924F91FD
:1033E0004F914F914F910895FF93EF93A0913E011C
:1033F000A0936E01AA270E94682EA0912C01A09391
:103400006A01A0910F01A0936D01A0912A01A093E0
:10341000690120922A01E8ECF1E0CCE2D7E0BEE2BB
:10342000AEE141914993AA95E1F7BA95C9F7EF91B9
:10343000FF910895FF93EF93A0916E010E94682E73
:10344000A0916D01A0930F01A0916A01A0932C019E
:10345000A0916901A0932A01ECE2F7E0C8ECD1E069
:10346000DECFA0910C01C6E0D4E0A9E4BFE441B1F5
:1034700058E040FDB99340FFA99346955A95C9F786
:10348000C4E2D4E0A0E3B1E340B158E040FDB99319
:1034900040FFA99346955A95C9F7C8EBD6E0AFEA25
:1034A000BFE241B158E040FDB99340FFA993469572
:1034B0005A95C9F7C6EDD6E0A0E8BEE440B158E0A1
:1034C00040FDB99340FFA99346955A95C9F70895D1
:1034D0000E944231130020494F2044495341424C3D
:1034E000454420000895452FA6E10E94B92E4F5B68
:1034F0000E94B42F4DE30E94B42FA7E10E94B92E81
:10350000C0E9DCE0C50FD21DC50FD21DA991B9914C
:103510009DE00E94D82E0895A3E10E945B31A5E0B2
:10352000C62FCA95AC9FCCEEDCE0C00DD11DA881A2
:10353000A7FF0AC00E944231FF43414C4C202000AB
:10354000A981AF770EC008950E944231FF464F52C5
:1035500020004A8146954F5B0E94B42F0E94B32FF2
:10356000A981BB27A39592E00E94D82E4AE30E942E
:10357000B42FBB27A881AF770E94D82E0895209240
:103580000F019927A7E00E94B92E0E94482F0E94A0
:10359000423112004249542030313233343536370B
:1035A00000000E9442311300444952000E944231FF
:1035B00014004C455600E8E9F8E30E94BE35A5E04A
:1035C0000E94B92E0E94423100004156522D43689C
:1035D0006970426173696332204D4F4E2020202074
:1035E0005000409137014F5C0E94B42F0E9442313D
:1035F000FF3A000092E0BB27AC2DA3950E94D82E85
:103600000E944231FF3A0000BB27AD2DA3950E94D6
:10361000D82EEBE7F1E0C6EED1E0AEE141EFB1919B
:10362000B03031F0BE8F4CAF4993AA95C1F706C0B8
:10363000B0E2BE8F4CAF4993AA95D1F7A7E10E94A3
:10364000B92EC0E0D4E0E1E1F0E10E9447329DE014
:1036500050E0452F4C5FB42FAA270E945B3143DF17
:1036600053955D30B1F7452F4950B42FA9E00E9422
:103670005B3139DF53955A31B1F7A7E30E94B92E78
:10368000C3E1D4E0EDE1F0E10E9447320E94423113
:103690000413535441434B3A00009927BB27A09190
:1036A00070010E94D82E6CE0C0917001C61720F006
:1036B000C61BB4E0B60F30DF6A95B1F708954F939B
:1036C0005F936F937F93EF93FF93CF93DF93AF93CA
:1036D000BF93AF92BF928F939F9386DED7DD4FDF6C
:1036E00031D08827A0912D014D3E11F4A16014C066
:1036F000413F11F4AA2710C0423F11F4A4600CC04E
:10370000433F39F497DE0E94A933AA270E94682E0E
:10371000E6CF443F29F71FC0A0932D014091160129
:103720004030E1F787DE9F918F91BF90AF90BF91BE
:10373000AF91DF91CF91FF91EF917F916F915F9169
:103740004F910895209217018CDE4091170140306F
:10375000D9F30C9449340E94B03370E0442425D04E
:10376000EAE7F8E30E94BE350E94A9334D3E11F40A
:10377000A160D2CF443F19F40E94B033B0CF463E8F
:1037800031F4703069F37A950E94B033E8CF473E48
:1037900031F47A3028F773950E94B033E0CF433F7D
:1037A000F9F643940E94B033DACFA7E00E94B92E15
:1037B0000E94482F0E94423100004156522D43681A
:1037C0006970426173696332204172726179205677
:1037D00069657700A0E60E94B92E0E94423102007E
:1037E000416472202000A0E50E94B92E0E9442315F
:1037F0000205202020202020202020446174612008
:1038000020202020202020202020000060E4679F2E
:10381000CCE3DDE0C00DD11DF00163E0A0E0B62FE8
:103820000E945B31A6E00E94B92EDF0191E00E9468
:10383000332FA5E0B62F0E945B31A5E00E94B92E80
:1038400090E058E0A991B0E00E94332F442D40FF52
:103850000BC0A7E10E94B92E219749910E94B42F75
:10386000A5E00E94B92E02C00E94B32F5A9551F7CD
:1038700038966395633191F60895204578697420F0
:10388000202020202020202020202020204368618C
:103890007220204D6F6E20202045786974202020F2
:1038A000476F20202053746570202056696577206B
:1038B00020417272617920922A0120923E01A5E096
:1038C0000E94B92EC0E0D0E0EDE1F6E10E94E532C1
:1038D000A0E50E94B92E0E944231010244464C41AB
:1038E00053482073697A653A20000E941F214F37A0
:1038F00049F40E944231FF353132204B69427974DC
:10390000650011C04F3F41F40E944231FF31204D0C
:1039100069427974650007C00E944231FF3020423D
:103920007974650013C00E9410214130D1F0E2E5A6
:10393000FBE3E8940E946B35413009F434C0453014
:1039400009F4B9CF423099F733D0B5CFEEE8FBE3B5
:10395000E8940E946B35413009F425C04530B1F739
:10396000AACFE6E1FBE3E8940E946B35413009F40D
:103970001AC0473019F40E94E51D9DCF4A3011F45A
:1039800017D099CF423011F46DD095CF433019F450
:103990000E943C1E90CF443019F40E948E1E8BCFA3
:1039A0004530F9F688CFA0911601A030E1F70895CF
:1039B0000E942E384F466F726D6174204D656469A8
:1039C000756D3F00413009F00895A6E20E94B92EBE
:1039D000C2E0D8E0EBE1FCE00E94AD320E9442314F
:1039E0000903466F726D617474696E672E2E2E2006
:1039F0002020202020000E9442310B0300000E9462
:103A00002221803001F50E9442310903466F726D18
:103A1000617474696E672E2E2E20446F6E652100CE
:103A2000A2E70E94B92E0E9442310B0320202050B1
:103A30007265737320616E79206B65792120200097
:103A40000E94A93308950E9442310903466F726DA6
:103A5000617474696E672E2E2E204572726F72210A
:103A60000000DECFA0E60E94B92EC4E0D8E0E9E174
:103A7000FDE00E94AD320E94423109054176616944
:103A80006C61626C653A00000E9442310A05466929
:103A90006C65733A20009CE00E940221DF93CF9373
:103AA000DF010E94D82E0E944231FF202F000E9489
:103AB0001F21A42FB0E011960E94D82E0E944231FF
:103AC0000B05426C6F636B733A00AF91BF910E941C
:103AD000D82E0E944231FF202F000E940A21A0EF21
:103AE000A49FD0011197B03009F413970E94D82EEB
:103AF000A6E00E94B92E0E9442310C0520202050E1
:103B00007265737320616E79206B657921202000C6
:103B10000E94A933089520457869742020496E6673
:103B20006F204261636B7570526573746F7252657A
:103B30007363616E20202020202044656C657465CD
:103B4000202020202020202020202020466F726D61
:103B50006174204578697420466F726D617420200D
:103B60002020202020202020202052657363616EB9
:103B70002020202020202020202020202020202045
:103B80002020202020202020202020202020204510
:103B90007869742020202020202020202020202030
:103BA00020202020202052657363616E2020202079
:103BB0002020202020202020202020202020202005
:103BC0002020202020202020202077270BD1A4E0B7
:103BD0000E94B92EC1E0D2E0ECE1F5E10E94E532AD
:103BE000A0E40E94B92E0E944231030244656C6534
:103BF00074652066696C6500B0D07093580105D378
:103C00004C3FD1F34CD1413019F4A72FB7D20ED38A
:103C100008957727E7D0A4E00E94B92EC1E0D2E052
:103C2000ECE1F5E10E94E532A0E40E94B92EA0E1AA
:103C3000A0935C010E9442310302536176652050DB
:103C40000000C7D28AD070935801DFD2403E20F4E2
:103C5000403161F0F4D0DECFD5D2D03021F4CC3079
:103C600010F427D1D7CF8AD2B4D108950CD14130E6
:103C700089F684D2BAD108957727B4D0A4E00E94FF
:103C8000B92EC1E0D2E0ECE1F5E10E94E532A0E41A
:103C90000E94B92EA2E1A0935C010E94423103026E
:103CA0004261636B7570000058D070935801ADD2BB
:103CB000403920F4423161F0C2D0DFCFA3D2D030FE
:103CC00021F4C03610F4F5D0D8CF58D21CD20895C4
:103CD000DAD0413091F652D222D20895772782D09D
:103CE000A4E00E94B92EC1E0D2E0ECE1F5E10E942F
:103CF000E532A0E40E94B92E0E94423103024C6FCB
:103D000061642050000065D228D0709358017DD2A4
:103D1000403111F0A2D0E3CF88D10895772762D047
:103D2000A4E00E94B92EC1E0D2E0ECE1F6E10E94ED
:103D3000E532A0E40E94B92E0E944231030252658E
:103D400073746F72650009D0709358015ED242316E
:103D500011F08ED0E4CFFBD108957727B5D00BD1E9
:103D60000E94A9334D3E21F42FD14F914F910895D8
:103D70004A3E09F40895403E19F40FD17727EECF5B
:103D8000413E21F40AD170916001E8CF443E49F4EC
:103D9000703031F302D17150472F4F704F30F1F234
:103DA000DECF453E59F440916001471709F4D8CF62
:103DB000F4D07395472F4F7089F2D1CF463E29F446
:103DC000703170F2EAD07051C9CF473E51F4409142
:103DD00060014F3031F04051471718F0DED0705F6E
:103DE000BDCFBECF0E941F21403019F44F914F919B
:103DF0001BC0409360010E9480330E94803310D228
:103E0000413019F04F914F9101C008950E9405383B
:103E10004F44464C415348206E6F7420666F726D5C
:103E200061747465640008950E9405384F44464CDF
:103E3000415348206572726F7221000008950E94FC
:103E400005384F43616E206E6F7420736176652074
:103E50006F6E20746869730008950E9405384F4E94
:103E60006F2042415349432066696C650000089504
:103E70000E9405384F4E6F204241434B55502066FB
:103E8000696C650008950E942E38C04F7665727780
:103E9000726974652066696C653F000008950E9430
:103EA0002E384F44656C6574652066696C653F000B
:103EB00008950E9405384F4E6F207370616365202E
:103EC0006C656674000008955F936F937F93A72FCE
:103ED000A07FA0936C01A0916C01AF70AB5FBA2F73
:103EE000A4E00E945B31A6E00E94B92EA0916C0173
:103EF000BB2795E00E94D82E0E94B32FA5E00E9418
:103F0000B92EA0916C01A09358017FD1ADD04F3F45
:103F100061F1A0916C01A093580140E040935A01D7
:103F200042E040935C01882784D1803091F4CCE357
:103F3000DFE00E94B32F5CE05F934991403808F0C6
:103F40004EE2403208F440E20E94B42F5F915A954D
:103F500099F7A0916C01A395A0936C01AF7009F043
:103F6000BACF7F916F915F9108955DE00E94B32F6A
:103F70005A95E1F7EECF4F935F93C4E1D5E0472F19
:103F80004F705EE1459FC00DD11D52EF47E159933F
:103F90004A95E9F75F914F9108954F935F93C4E17C
:103FA000D5E0472F4F705EE1459FC00DD11D5CE00D
:103FB00044E059934A95E9F75AE043E159934A9509
:103FC000E9F75F914F910895A0911601A030E1F7B4
:103FD0000895709358014CE040935A0140E140939A
:103FE0005C0121D1803009F01FCF7093580190916E
:103FF0003D01E0E0F0E99770929540EC949FE00D70
:10400000F11D40E04F9300E0CCE3DFE01591199300
:104010000A95E1F740935A0142E040935C010CD1CC
:104020004F9143954C3071F7089590913D019770F1
:10403000E0E0F0E9929540EC949FE00DF11D40E046
:104040004F9340935A0142E040935C0170935801B2
:10405000F0D0CCE3DFE00E947A7932964F9143951D
:104060004C3071F778940895403139F40E94423110
:10407000FF4241533A0040E10895423139F40E9431
:104080004231FF4255503A0042E10895443139F43B
:104090000E944231FF5553523A0044E1089546319F
:1040A00039F40E944231FF4348383A0046E108950E
:1040B000483139F40E944231FF4156523A0048E1FA
:1040C00008954A3139F40E944231FF47504F3A0077
:1040D0004AE108954C3139F40E944231FF53414D79
:1040E0003A004CE108954E3139F40E944231FF4CC0
:1040F000424C3A004EE108950E944231FF2D2D2D91
:104100002D004FEF08957093580140E640935A01F7
:1041100042E140935C0187D0803009F085CE7093F6
:1041200058014427E0E0F0E94F93CCE3DFE00024BE
:10413000159019920A94E1F740935A0142E0409396
:104140005C017AD04F914395403671F7089540E075
:10415000E0E0F0E94F9340935A0142E040935C0164
:104160007093580166D0CCE3DFE00E947A793296F2
:104170004F914395403671F7789408954F93FF938C
:10418000EF93DF93CF93BF93AF9340912C01409374
:1041900061014CE440932C01C6E0DAE0E7E1FCE089
:1041A0000E94AD320E9442310B0757726974696EEA
:1041B0006720646174612E2E2E004091610140934E
:1041C0002C01AF91BF91CF91DF91EF91FF914F9172
:1041D0000895CAE2CAE240913D01942F4F5C499391
:1041E00040E249934BE54993409129014F93406840
:1041F000409329010E94AC794DE549934F9140933A
:10420000290108950E94C83C08950E94943D0E948F
:10421000573B08950E94043B08950E94843B0895F3
:104220000E94A33C08950E94293D08950E949C3D50
:1042300008950E941C3E08950E94BD3D08950E946D
:10424000123B08950E94353C0895A1E00E94243558
:1042500020922A0120923E01A7E00E94B92EC0E0E0
:10426000D0E0EDE1F6E10E94E532A0E70E94B92E30
:104270000E94423101024156522D436869704261E9
:104280007369633220636F6E66696770616765008A
:10429000A7E00E94B92E0E94423114014368656371
:1042A0006B73756D3A20000088D15ED092D0C4D077
:1042B000F5D026D14CD1ECE1F6E4E8940E946B35C0
:1042C000413009F475C1423059F440910C0151E07C
:1042D000452740930C010E9407790E94D822E5CF20
:1042E000433059F440910C0152E0452740930C01B2
:1042F0000E9407790E94D822D8CF443059F44091C7
:104300000C0154E0452740930C010E9407790E945C
:10431000D822CBCF453059F440910C0158E04527C5
:1043200040930C010E9407790E94D822BECF4730EB
:1043300049F40E941A79439547700E9415790E94AA
:10434000D822B3CF483059F440910C0150E14527B1
:1043500040930C010E9407790E94D822A6CF4A30D0
:1043600011F40E942E2B71CFA6E00E94B92E0E945C
:10437000423103014B6579626F617264206C61792F
:104380006F75743A0000A7E040910C01417009F488
:10439000A1E70E94B92E0E94423103124445202811
:1043A00051574552545A2900A7E040910C014170E1
:1043B00009F0A1E70E94B92E0E9442310412555320
:1043C00020285157455254592900A7E00E94B92E80
:1043D0000895A6E00E94B92E0E944231060153655D
:1043E0007269616C2073706565643A00A7E0409162
:1043F0000C01427009F4A1E70E94B92E0E944231DB
:104400000612203132303020427073202000A7E0A5
:1044100040910C01427009F0A1E70E94B92E0E9460
:104420004231071220323430302042707320200095
:10443000A7E00E94B92E0895A6E00E94B92E0E941E
:10444000423109014932432073706565643A0000C6
:10445000A7E040910C01447009F4A1E70E94B92E35
:104460000E94423109122020313030206B487A20DE
:104470002000A7E040910C01447009F0A1E70E94E0
:10448000B92E0E9442310A122020343030206B486D
:104490007A202000A7E00E94B92E0895A6E00E948D
:1044A000B92E0E9442310C0153504920737065654A
:1044B000643A0000A7E040910C01487009F4A1E7BC
:1044C0000E94B92E0E9442310C122020202035205B
:1044D0004D487A202000A7E040910C01487009F077
:1044E000A1E70E94B92E0E9442310D1220203135E1
:1044F00036206B487A202000A7E00E94B92E08954C
:10450000A6E00E94B92E0E9442310F01454550524B
:104510004F4D20616464726573733A00A1E70E9495
:10452000B92E0E9442310F122020202020000E942C
:104530001A794770405D0E94B42F0E944231FF20DB
:10454000202020200000A0E70E94B92E0895A6E0B8
:104550000E94B92E0E94423111014C696E652045BE
:104560006E643A00A7E040910C01407109F4A1E7A4
:104570000E94B92E0E944231111220202043522B5A
:104580004C4620202000A7E040910C01407109F02A
:10459000A1E70E94B92E0E944231121220206F6EB4
:1045A0006C79204C46202000A7E00E94B92E089587
:1045B000A0911601A030E1F70895AA27BB27CC27C8
:1045C000DD27EE27FF27159042E0149EA00DB11DB8
:1045D000C21DD21D459147E0149EA00DB11DC21D04
:1045E000D21DFE3881F7EE27F0EF459141E7149E8A
:1045F000B01DC11DD21D459147E0149EB01DC11DC7
:10460000D21DF03091F7BF93AF93DE019FE00E947F
:10461000332FAF91BF910E94332F089520457869C1
:104620007420204B65796220205365722020204938
:1046300032432020205350492020202020202020B9
:10464000454550524F4D204C696E6520202020205A
:104650002020436C6F6E6520AEE0A0932C01C1E07A
:10466000D4E0ECE1F2E10E94AD320E944231050556
:1046700000000E943C020E944231060320202020BC
:104680002028632920323030362D32303039202036
:104690002020202000000E944231070320202020FB
:1046A0006279204A6F65726720576F6C6672616D20
:1046B000202020200000A2EAA0932C010E94423179
:1046C000090320202020202044656469636174650B
:1046D0006420746F20202020202000000E9442319E
:1046E0000A03466C6F7269616E2C204572696B20FB
:1046F000616E64204469616E612E0000AEE0A0939B
:104700002C010E9442310C025468697320736F6659
:104710007477617265206973206C6963656E736577
:1047200064000E9442310D04756E646572207468E5
:1047300065207465726D73206F6620746865200053
:104740000E9442310E04474E55205055424C494379
:10475000204C4943454E534520562E3220000E949E
:1047600042310F0355736520697420617420796F9D
:104770007572206F776E207269736B210000A2EC56
:10478000A0932C010E9442311107205052455353EF
:1047900020414E59204B455920000E94A9330895CD
:1047A00061E00E945435509116015D3E09F4089570
:1047B0004531B1F790913D01E0E0F0E997709295B5
:1047C00040EC949FE00DF11DCCE3DDE050E045911D
:1047D00049935A95E1F7CCE3DDE00E94233A0E9429
:1047E0005435509116015D3E11F34630A1F76395A3
:1047F000CCEBDDE00E94233A0E9454355091160123
:104800005D3EA9F24630A1F763956931E9F644E0CF
:104810000E943835089590913D019770E0E0F0E9ED
:10482000929540EC949FE00DF11D45E10E943835D2
:1048300060E06F93CCE3DFE00E94003A803041F00B
:10484000813051F1883241F145E10E943835F2CF93
:1048500046E00E943835CCEBDFE00E94003A803021
:1048600041F08130C9F08832B9F045E10E94383515
:10487000F2CF0E947A797894329646E00E943835D9
:104880006F9163956C30A9F60E9444354430E1F78E
:1048900046E00E94383508956F91089561E00E94C6
:1048A0005435509116015D3E09F408954531B1F734
:1048B000A0E8762F7A95A79FE001ACE3BDE070E811
:1048C0000E94B63A4D937A95D9F7CCE3DDE00E9489
:1048D000233A0E945435509116015D3E31F3463023
:1048E000A1F763956F3021F744E00E9438350895B1
:1048F00045E10E94383560E06F93CCE3DDE00E9433
:10490000003A803031F0883201F145E10E943835BB
:10491000F4CFA0E8762F7A95A79FE001ACE3BDE045
:1049200070E84D910E94BF3A7A95D9F746E00E940F
:1049300038356F9163956E30F9F60E9444354430F6
:10494000E1F746E00E94383508956F9108950241DD
:104950004253282E2E2E0353474E282E2E2E04531C
:104960005152282E2E2E054E4F54282E2E2E0652F2
:104970004E44282E2E2E07414443282E2E2E084921
:104980004E282E2E2E2E09585045454B282E0A54BF
:10499000454D50282E2E0B4C4F282E2E2E2E0C48D7
:1049A00049282E2E2E2E0D4B4559282E2E2E0E45E3
:1049B0005045454B282E0F455252282E2E2E104181
:1049C00052282E2E2E2E1153494E282E2E2E1243B3
:1049D0004F53282E2E2E134654595045282E144638
:1049E00053495A45282E155053544154282E1653D6
:1049F0005049282E2E2E174D454E55282E2E8050CC
:104A000052494E542E2E81434C532E2E2E2E824729
:104A10004F544F2E2E2E83424F582E2E2E2E844131
:104A2000434F50592E2E8553594E432E2E2E8645D8
:104A30004E442E2E2E2E8742434F50592E2E8854F0
:104A400048454E2E2E2E89504F532E2E2E2E8A4EF6
:104A50004F54452E2E2E8B454D49542E2E2E8C52C2
:104A6000524541442E2E8D5257524954452E8E4761
:104A70004F5355422E2E8F52455455524E2E90561E
:104A80004D4F44452E2E914E4558542E2E2E924970
:104A90004E5055542E2E93504C4F542E2E2E94572C
:104AA0004149542E2E2E95545345542E2E2E965455
:104AB0004745542E2E2E974653454C454354984F08
:104AC0004E4552522E2E99535055542E2E2E9A53F7
:104AD0004745542E2E2E9B45504F4B452E2E9C471E
:104AE00045545049582E9D434952434C452E9E43B0
:104AF0004F4C4F522E2E9F424F524445522EA046AD
:104B00004F4E542E2E2EA150554D502E2E2EA258C3
:104B1000504F4B452E2EA359454D49542E2EA44C93
:104B2000494D49542E2EA547455443484152A64469
:104B3000524157544F2EA7504C41592E2E2EA85358
:104B400050524954452EA95343524F4C4C2EAA4221
:104B50005245414B2E2EAB464153542E2E2EAC5374
:104B60004C4F572E2E2EAD445241572E2E2EAE496D
:104B7000434F4D4D2E2EAF444154412E2E2EB04367
:104B8000544558542E2EB146524541442E2EB2461D
:104B900057524954452EB343424F582E2E2EB447F8
:104BA000455441545452B54644454C455445B64687
:104BB000424F582E2E2EB750414C45545445B846BE
:104BC0004F522E2E2E2EB949462E2E2E2E2EBA4460
:104BD00049522E2E2E2EBB4F55542E2E2E2EBC4615
:104BE000434952434C45BD414C4552542E2EBE467E
:104BF000435245415445BF41534B2E2E2E2EC03FAC
:104C00002E2E2E2E2E2EC742432E2E2E2E2ECA4E46
:104C10004F2E2E2E2E2ECB454D2E2E2E2E2ECC52FE
:104C200052442E2E2E2ECD5257522E2E2E2ECE47A1
:104C30004F532E2E2E2ECF5245542E2E2E2EC2479F
:104C40004F2E2E2E2E2ED0564D2E2E2E2E2ED249BB
:104C50004E502E2E2E2ED3504C2E2E2E2E2ED7468C
:104C600053454C2E2E2EDC4750582E2E2E2EDD4333
:104C7000492E2E2E2E2EDE434F4C2E2E2E2EDF4270
:104C80004F2E2E2E2E2EE44C494D2E2E2E2EE54745
:104C900043482E2E2E2EE644544F2E2E2E2EE85311
:104CA00050522E2E2E2EED44522E2E2E2E2EEE490A
:104CB000432E2E2E2E2EEF44412E2E2E2E2EF1463A
:104CC00052442E2E2E2EF24657522E2E2E2EF447C2
:104CD00041542E2E2E2EF54644454C2E2E2EF750A6
:104CE000414C2E2E2E2EFC4643492E2E2E2EFE46B5
:104CF00043522E2E2E2E002E2E2E2E2E2E2EA091F4
:104D00000801B0910901ED01E2EBF2E0CE0FDF1FE7
:104D1000F6EFE0910E01FE0F7F934F92EEE14E2EE3
:104D20006991ED915491762F7295762757FD6727FB
:104D300068B9ED91000056FD76B9049055FD76B93D
:104D40006991162E54FD76B91294162653FD76B944
:104D500007FC61254A9452FD76B9502D712D41F71B
:104D600060910F0168B94F907F91EE91F0910E0123
:104D7000F395FA3029F4FF27A0930801B0930901B5
:104D8000F0930E010C94672DA0910801B0910901D8
:104D9000D0910001C0910101C295DC0FDE7EE5E1FA
:104DA00010900F01FD914D2FF0FD429548B9000084
:104DB0004D2FF1FD429548B900004D2FF2FD42956F
:104DC00048B900004D2FF3FD4295000048B96D2F02
:104DD0004D2FF4FD429548B9CD91F5FD62955D2FBB
:104DE00068B9F6FD52956D2F4D2F58B9F7FD6295B4
:104DF000C0FD4295000068B9FC2FEA95B9F618B8D5
:104E0000EE91F0910E01F395F23029F4FF27A09373
:104E10000801B0930901F0930E010C94672DA09145
:104E20000801B0910901D1E0FEE110900F01ED9170
:104E3000CE2FC370588158B9CE2FC695C695C37072
:104E40005881E29558B9CE2FC3705881CE2FC695A0
:104E500058B9C695C3705881ED91CE2F58B9C3701B
:104E60005881FA9541F718B8EE91F0910E01F3953B
:104E7000F33029F4FF27A0930801B0930901F093C0
:104E80000E010C94672DA0910801B09109010F93B8
:104E900010900F01EAE2D1E0CD91C6950C2FC2959A
:104EA000C770F881F8B9C02F0000C770F881000002
:104EB00000000000F8B9CD91C6950C2FC295C770BF
:104EC000F881EA9579F718B811970F91F0910E01D2
:104ED000F395F43029F4FF27A0930801B09309015A
:104EE000F0930E010C94672DA0910801B091090177
:104EF000D0910001C0910101C295DC0FDE7EE0E19E
:104F000010900F01FD914D2FF0FD429548B9000022
:104F1000000000004D2FF1FD429548B9000000004F
:104F200000004D2FF2FD429548B9000000004D2FC2
:104F3000F3FD4295000048B9000000006D2F4D2F91
:104F4000F4FD429548B90000CD91F5FD62955D2FC5
:104F500068B900000000F6FD52956D2F4D2F58B92D
:104F6000F7FD6295C0FD42950000000068B9FC2F76
:104F700000000000EA9551F6000018B8EE91F0919B
:104F80000E01F395F33029F4FF27A0930801B093A5
:104F90000901F0930E010C94672DA0910801B091C6
:104FA0000901C0914101D82DF6EFE0910E01FE0FED
:104FB000E395E0930E01EA3088F1EC3069F59396C1
:104FC000A0930801B093090120920E01DC3031F466
:104FD000D0914001D09341010C94672DD83189F4D0
:104FE000A1E3B2E0C0912E01D3E2CD9FA00DB11D8F
:104FF000CFE0A0930801B0930901C09341010C9444
:10500000672DD83D49F4CBE4AEE0B2E0A0930801AF
:10501000B0930901C09341010C94672D0F931F9326
:105020002F93D83D28F4DC2F0C2F1C2F2C2F05C0DC
:1050300029E61DE208E8DCECCBE46C2F7C2F7295AE
:10504000ED91E7FD6727EF775491ED9168B9172E41
:1050500056FD16B86C2F7C2F729555FD16B8E7FDDE
:10506000672754FD16B8EF77000053FD16B804907B
:1050700052FD16B8502DED9168B9172E56FD16B891
:105080006C2F7C2F729555FD16B8E7FD672754FDF0
:1050900016B8EF77000053FD16B8049052FD16B80D
:1050A000502DED9168B9172E56FD16B86C2F7C2F38
:1050B000729555FD16B8E7FD672754FD16B8EF77D2
:1050C000000053FD16B8049052FD16B8502DED9116
:1050D00068B9172E56FD16B86C2F7C2F729555FDAA
:1050E00016B8E7FD672754FD16B8EF77000053FDAB
:1050F00016B8049052FD16B8502DED9168B9172ED0
:1051000056FD16B86C2F7C2F729555FD16B8E7FD2D
:10511000672754FD16B8EF77000053FD16B80490CA
:1051200052FD16B8502DED9168B9172E56FD16B8E0
:105130006C2F7C2F729555FD16B8E7FD672754FD3F
:1051400016B8EF77000053FD16B8049052FD16B85C
:10515000502DED9168B9172E56FD16B86D2F7D2F85
:10516000729555FD16B8E7FD672754FD16B8EF7721
:10517000000053FD16B8049052FD16B8502DED9165
:1051800068B9172E56FD16B86D2F7D2F729555FDF7
:1051900016B8E7FD672754FD16B8EF77000053FDFA
:1051A00016B8049052FD16B8502DED9168B9172E1F
:1051B00056FD16B86D2F7D2F729555FD16B8E7FD7B
:1051C000672754FD16B8EF77000053FD16B804901A
:1051D00052FD16B8502DED9168B9172E56FD16B830
:1051E0006D2F7D2F729555FD16B8E7FD672754FD8D
:1051F00016B8EF77000053FD16B8049052FD16B8AC
:10520000502DED9168B9172E56FD16B86D2F7D2FD4
:10521000729555FD16B8E7FD672754FD16B8EF7770
:10522000000053FD16B8049052FD16B8502DED91B4
:1052300068B9172E56FD16B86D2F7D2F729555FD46
:1052400016B8E7FD672754FD16B8EF77000053FD49
:1052500016B8049052FD16B8502DED9168B9172E6E
:1052600056FD16B86D2F7D2F729555FD16B8E7FDCA
:10527000672754FD16B8EF77000053FD16B8049069
:1052800052FD16B8502DED9168B9172E56FD16B87F
:10529000602F702F729555FD16B8E7FD672754FDF6
:1052A00016B8EF77000053FD16B8049052FD16B8FB
:1052B000502DED9168B9172E56FD16B8602F702F3E
:1052C000729555FD16B8E7FD672754FD16B8EF77C0
:1052D000000053FD16B8049052FD16B8502DED9104
:1052E00068B9172E56FD16B8602F702F729555FDB0
:1052F00016B8E7FD672754FD16B8EF77000053FD99
:1053000016B8049052FD16B8502DED9168B9172EBD
:1053100056FD16B8602F702F729555FD16B8E7FD33
:10532000672754FD16B8EF77000053FD16B80490B8
:1053300052FD16B8502DED9168B9172E56FD16B8CE
:10534000602F702F729555FD16B8E7FD672754FD45
:1053500016B8EF77000053FD16B8049052FD16B84A
:10536000502DED9168B9172E56FD16B8602F702F8D
:10537000729555FD16B8E7FD672754FD16B8EF770F
:10538000000053FD16B8049052FD16B8502DED9153
:1053900068B9172E56FD16B8612F712F729555FDFD
:1053A00016B8E7FD672754FD16B8EF77000053FDE8
:1053B00016B8049052FD16B8502DED9168B9172E0D
:1053C00056FD16B8612F712F729555FD16B8E7FD81
:1053D000672754FD16B8EF77000053FD16B8049008
:1053E00052FD16B8502DED9168B9172E56FD16B81E
:1053F000612F712F729555FD16B8E7FD672754FD93
:1054000016B8EF77000053FD16B8049052FD16B899
:10541000502DED9168B9172E56FD16B8612F712FDA
:10542000729555FD16B8E7FD672754FD16B8EF775E
:10543000000053FD16B8049052FD16B8502DED91A2
:1054400068B9172E56FD16B8612F712F729555FD4C
:1054500016B8E7FD672754FD16B8EF77000053FD37
:1054600016B8049052FD16B8502DED9168B9172E5C
:1054700056FD16B8612F712F729555FD16B8E7FDD0
:10548000672754FD16B8EF77000053FD16B8049057
:1054900052FD16B8502DED9168B9172E56FD16B86D
:1054A000612F712F729555FD16B8E7FD672754FDE2
:1054B00016B8EF77000053FD16B8049052FD16B8E9
:1054C000502DED9168B9172E56FD16B8612F712F2A
:1054D000729555FD16B8E7FD672754FD16B8EF77AE
:1054E000000053FD16B8049052FD16B8502DED91F2
:1054F00068B9172E56FD16B8622F722F729555FD9A
:1055000016B8E7FD672754FD16B8EF77000053FD86
:1055100016B8049052FD16B8502DED9168B9172EAB
:1055200056FD16B8622F722F729555FD16B8E7FD1D
:10553000672754FD16B8EF77000053FD16B80490A6
:1055400052FD16B8502DED9168B9172E56FD16B8BC
:10555000622F722F729555FD16B8E7FD672754FD2F
:1055600016B8EF77000053FD16B8049052FD16B838
:10557000502DED9168B9172E56FD16B8622F722F77
:10558000729555FD16B8E7FD672754FD16B8EF77FD
:10559000000053FD16B8049052FD16B8502DED9141
:1055A00068B9172E56FD16B8622F722F729555FDE9
:1055B00016B8E7FD672754FD16B8EF77000053FDD6
:1055C00016B8049052FD16B8502DED9168B9172EFB
:1055D00056FD16B8622F722F729555FD16B8E7FD6D
:1055E000672754FD16B8EF77000053FD16B80490F6
:1055F00052FD16B8502DED9168B9172E56FD16B80C
:10560000622F722F729555FD16B8E7FD672754FD7E
:1056100016B8EF77000053FD16B8049052FD16B887
:10562000502DED9168B9172E56FD16B8622F722FC6
:10563000729555FD16B8E7FD672754FD16B8EF774C
:10564000000053FD16B8049052FD16B8502DED9190
:1056500028B82F911F910F910C94672D0E942E381E
:105660006F436C6F6E652073797374656D3F2000B6
:10567000413009F0089565D087D0803079F078D036
:105680000E9405384F4E6F20636F6E74726F6C6CA2
:10569000657220666F756E64200008958DD080302D
:1056A00069F066D00E9405384F4E6F204D656761E6
:1056B00036343420666F756E64000895CDD09DD069
:1056C000EE27FF2750E060E00590B8D00590BDD0F0
:1056D00063956038C9F79ED05395A9F74CEA4ED030
:1056E00040EA4CD04AD046EE49D00E9480330E9416
:1056F00080330E9480334CEA41D048EA3FD03DD00D
:1057000041ED3CD00E9480330E9480330E94803360
:105710004CEA34D044EA32D030D04CEF2FD00E9443
:1057200080330E9480330E94803322D00E9405384B
:105730008053797374656D20636C6F6E65640000CF
:10574000089543E54CBD2DBC249A2C984FEF4A9503
:10575000F1F72C9A4FEF4A95F1F72C984FEF4A95B5
:10576000F1F72C984FEF4A95F1F70E948033089596
:105770002C9A4CE54CBD3DBC089544274EBD4DB51B
:1057800047FFFDCF4EB5089588274CEAF7DF43E584
:10579000F5DFF3DF433509F081E0EFDF0895BF93D4
:1057A000AF934F93A42FBB270E94332F0E94B32F98
:1057B0004F91AF91BF910895882740E3DFDFDDDF90
:1057C00040E0DCDFDADF4E3111F082E0089540E3A3
:1057D000D5DFD3DF41E0D2DFD0DF463911F082E000
:1057E000089540E3CBDFC9DF42E0C8DFC6DF4930C0
:1057F00019F04A3009F082E008954CEABFDF40E832
:10580000BDDFBBDFBADF0E9480330E9480330E947D
:10581000803308954CE4B2DF452F4695AFDF452F26
:10582000440F440F440F440F440F440F440FA6DFAE
:10583000A4DF0E9480330E948033089540E49EDFFD
:105840009CDF462F9BDF402D99CF48E497DF95DF03
:10585000462F94DF402D92CF4F93FF93EF93DF932A
:10586000CF93BF93AF9340912C01409361014CE4DF
:1058700040932C01C5E0DAE0E8E1FCE00E94AD32A3
:105880000E9442310B06436C6F6E696E672053793C
:105890007374656D2E2E2E004091610140932C0192
:1058A000AF91BF91CF91DF91EF91FF914F9108950B
:1058B00028B818954F935F936F93FF93EF93DF93FF
:1058C000CF93BF93AF930F921F92FFB7FF93309286
:1058D0001101B0913101B7FF5C98B7FD5C9A4B990B
:1058E000BE7F4B9BB160B0933101C8E0D1E05F89CE
:1058F000A889E9890A881B88A00DE11DA88BE98B7E
:10590000FFA14491AD89AF3F09F4452F5AA5450346
:10591000B0E8B10DB093B300EE89FF89488D598D81
:10592000AA27E2FDA095E5FDA095F4FDA09557FD01
:10593000A095AA1FEE1FFF1F441F551FEE8BFF8B64
:10594000488F598F830C921CEBA9FF81EF23E8B994
:105950007894E9A190FC04C0F8A58F1608F490C0D3
:10596000FCE0E2FFFDEE8F1639F45E98E3FFAFC076
:10597000B2E8B0938000ABC0F1E1E2FFF3EF8F1625
:1059800039F45E9AE3FFA3C0B2ECB09380009FC0ED
:10599000FBE1E2FFFFEF8F1621F4EFEFE0933B0115
:1059A00096C0F2E0E2FFF9EE8F1619F420923B0167
:1059B0008EC0F9E3E2FFF7E08F1609F088C0A8EC8B
:1059C000A883A1E0A9832E8288249924AAE0A9AF04
:1059D000A5E0E2FFA39542E3E2FF4CE3BA8DB39565
:1059E000BA1731F4BB27EB8DFC8D3196EB8FFC8F12
:1059F000BA8FE885E395E41709F4EE27E887FDE818
:105A0000E0E0AC89EA0FF21DB491B21511F0A39554
:105A1000AC8BBAA7A0915001A03009F458C0B09146
:105A20005101B395B0935101BA17C0F3BB27B0939E
:105A30005101E0915201F0915301C0915601D09172
:105A400057012196A191E0935201F0935301AE3F8B
:105A500009F05FD6FD1798F0EC1788F0A09133019C
:105A6000A13029F4A2E020925001A0933301E091EB
:105A70005401F0915501E0935201F093530127C076
:105A8000A0918400AA3FE0F3AB3F00F0AC3F00F0F0
:105A9000AD3F00F0AE3F00F0E5FD19C0E0912901F7
:105AA000E7FD0C94CD27E0913E01E53011F40C9414
:105AB0007427E37011F40C947F26E13011F40C94F8
:105AC000C426E23011F40C940F270C944327A091C4
:105AD0001401A5FD25C0E091C000E7FF69C0E09179
:105AE000C600F5EFB491B0FF36C0A7FF03C0209207
:105AF00016015BC0E33809F4E0E1F6E840910C01DF
:105B000040FDFE5FEF77A4FFA6FDF395A4FFA0FD87
:105B1000E068A1FDE068E491E0931501A06246C051
:105B2000E0911501E0931601E0931701EE3E19F4A0
:105B3000A2FD0C94380040912D01E33611F4A2FD32
:105B40004160E03711F4A3FD4260EC3F09F444608A
:105B500040932D012AC0E03F11F4A06827C0E03E29
:105B600011F4A06423C0E23131F4A6FD1EC0A1608F
:105B7000A7FDAE7F1AC0E93521F4A260A7FDAD7F75
:105B800014C0E43151F4A6FD04C0A460A7FDAB7FAE
:105B90000CC0A860A7FDA77F08C0E13121F4A06177
:105BA000A7FDAF7E02C020921601AF71A093140131
:105BB00040910C0141FD0E94A17841FF0E94D678DE
:105BC000FF91FFBF1F900F90AF91BF91CF91DF91D9
:105BD000EF91FF916F915F914F911895AAEBA4B946
:105BE000AFEFA5B9A0EEA7B9A0E0A8B9A0EFAAB9F8
:105BF000AFEFABB9A6B1AF77A0932901B2ECB093E8
:105C00008000B9E1B0938100F4E0A2FFF4E0F093EA
:105C10008700FEEFA2FFF6EFF09386002092890046
:105C2000FAE5F0938800F4E0F0938B00F8EDF09340
:105C30008A00A6E0A0936F00A2E0A4BDA1E0A5BDEC
:105C4000A1E3A7BDA3E8A093B000A1E0A093B10099
:105C5000A0E8A093B3002092B6002092C000A0E17B
:105C6000A093C100A6E6A093C200ACE5B0910C01E0
:105C7000B3FDAFE5ACBDA0E0ADBDA5E17AD0C8E015
:105C8000D1E0A8ECA993A1E0A993AEE12992AA954D
:105C9000E9F7AAEAA0931E01A093200120922A010D
:105CA00020920D01AEE3A0931C010F9300912901F6
:105CB0000F770093290106EE07C00F930091290189
:105CC00000680093290104EE009330010F910895BC
:105CD000A0933E01A03041F4ACE3A0934401AEE2B6
:105CE000A0934501A6EE42C0A13069F4A8EAA093B2
:105CF0004401A4E7A0934501A0E0A0930001A0EE19
:105D0000A093010124C0A23091F4A8E7A09344011C
:105D1000ACE4A0934501C0E0D1E0A0E0A993A0E4E9
:105D2000A993A0EAA993A0EEA993A3EE1FC0A33064
:105D300081F4A4E5A0934401AAE3A0934501C0E047
:105D4000D1E0AA27B8E0A993A05EBA95E1F7A7EE43
:105D50000DC0A0E8A0934401A0E4A0934501A0E2F7
:105D6000A0930001A0EEA0930101A0ECA09330014C
:105D70000895AA0FAE7EA0932C010895A295AA0FB4
:105D8000A07EA0930F01089548834091290147FD0B
:105D90000EC0CF93DF935F9342EBC40F42E0D41F5A
:105DA00040912C014E7E48835F91DF91CF91089501
:105DB0004F935F936F93AF93BF9340E2592F53700C
:105DC000523061F0533009F44BE2B7FF05C0A095A3
:105DD000B095A30DB21D4DE20E94B42F592F5C70F7
:105DE000692F6073E8944FE24395A051B742E0F702
:105DF000A05FB84D5C3009F42BD04FE24395A85E0C
:105E0000B340E0F7A851BC4F53FD22D0603309F4F2
:105E1000A8D04FE24395A456B209E0F7AC59BF4F62
:105E2000503009F015D0603209F49BD04FE2439511
:105E3000AA50E8F70DD0A65F603109F492D040E394
:105E40004A0F92D0BF91AF916F915F914F9108959A
:105E5000403311F0689488C091FD86C0F6F390FF3E
:105E6000089581C008954F9390FF05C04B2F429530
:105E700009D04B2F07D04A2F429504D04A2F02D089
:105E80004F9108954F70405D4A3308F0495F6CC0F0
:105E900040913E014030B1F0AF93BF93CF93DF9379
:105EA000D1E0C8ECACE5BEE12992BA95E9F7AA9534
:105EB000D1F7DF91CF91AA24BB2420922B01BF916F
:105EC000AF910895AF93BF93CF93DF9340E2D1E0BA
:105ED000C8ECA7E1BEE14993BA95E9F7AA95D1F7D5
:105EE00040912C014E7EA7E1BEE14993BA95E9F7B6
:105EF000AA95D1F7DF91CF91AA24BB2420922B0140
:105F0000BF91AF910895AF93BF9320922B01A091C1
:105F10002A01A03051F4A7E1AA24B394AB1571F77C
:105F2000B6E1BB2ECF93DF9366C0A13021F4BF91C1
:105F3000AF910C942C35A23049F44DE0B0910C0196
:105F4000B4FF94D4BF91AF914AE090C4A33019F448
:105F5000BF91AF910895BF91AF915AE00E94463A28
:105F600008954CE201C040E2AF93BF93A0912B0192
:105F7000A395A0932B01A0912A01A43030F0BF91EA
:105F8000AF91542F0E94463A0895A030A9F0A33053
:105F900059F4A42FBB275F936F930E94C0176F9192
:105FA0005F91BF91AF910895BF91AF91A0912A01E8
:105FB000A1FF0C9438355AC4EF93E0913E01E030D4
:105FC00009F09AC0EF91CF93DF932FD496FD35C09F
:105FD000DBDEA395AE3131F4AA27B395B73111F4C6
:105FE000B6E107C0AA2EBB2EDF91CF91BF91AF9132
:105FF0000895AA2EBB2ED1E0C8EC4F93A6E1BEE1D6
:106000004E8D4993BA95E1F7AA95C9F7AEE140E202
:106010004993AA95E9F7D4E0CAE7A6E1BEE14E8D1F
:106020004993BA95E1F7AA95C9F7AEE140912C01E1
:106030004993AA95E9F74F91D7CFAB31A8F6B23182
:1060400098F6AD5FAA2EEF93FF934F925F926F92F7
:106050007F9270F85F93E42FF6EFB5E04424552467
:1060600066245527A491A7FD539550FB40F8A6FD43
:10607000539550FB41F8A5FD539550FB50F8A4FDF6
:10608000539550FB51F8A3FD539550FB60F8A2FDCA
:10609000539550FB61F8F3955527A491A7FD5395AF
:1060A00050FB42F8A6FD539550FB43F8A5FD5395D0
:1060B00050FB52F8A4FD539550FB53F8A3FD5395A4
:1060C00050FB62F8A2FD539550FB63F8F395442D05
:1060D0005BDE2196452D58DE2196462D55DE6C96C9
:1060E000BA9509F0BBCF5F9170FA7F906F905F9087
:1060F0004F90FF91EF9178CFFF93CF93DF936F9302
:106100007F93E42F60910D0160FD1EC0F6EFAA2D74
:10611000BB2DDAE0C49137D0B395AA2D96FD33D0CC
:1061200096FDB395F395AA2DDA95A1F7AA2DAA5F4E
:1061300096FDAA5FAA2E7F916F91DF91CF91FF917B
:10614000EF91BF91AF910895FCE7EF77AE2FEEEEA0
:10615000EA0FF21DAA0FEA0FF21DAA2DBB2DD6E001
:10616000C49155D0B395AA2D96FD51D096FDB39507
:10617000D0FD3196AA2DDA9599F7AA2DAC5F96FD40
:10618000AC5FAA2ED8CF60912C016F936295C7FDAA
:10619000629560932C01A2D0A39596FD9FD096FDA9
:1061A000A395C6FD629560932C0198D0A39596FDAA
:1061B00095D096FDA395C5FD629560932C018ED078
:1061C000A39596FD8BD096FDA395C4FD6295609333
:1061D0002C0184D0A39596FD81D096FDA395C3FD97
:1061E000629560932C017AD0A39596FD77D096FDA9
:1061F000A395C2FD629560932C0170D0A39596FD86
:106200006DD096FDA3956F9160932C0108956091D8
:106210002C01D0FDC295762FC7FF729570932C018B
:106220005DD0A39596FD5AD096FDA395762FC6FF17
:10623000729570932C0152D0A39596FD4FD096FD88
:10624000A395762FC5FF729570932C0147D0A39527
:1062500096FD44D096FDA395762FC4FF729570935A
:106260002C013CD0A39596FD39D096FDA395609363
:106270002C0108954F934591403011F44F910895AA
:1062800073DEF9CFFF91EF91EE0FFF1FAF93BF9336
:10629000B591BF3F11F0A5910ED0BF91AF914F9333
:1062A0004591403031F44F913197F695E79531960D
:1062B00009945ADEF5CFEF93E0913E01E03021F0F2
:1062C000EF91AA2EBB2E0895EF91AE3108F0ADE10B
:1062D000B73108F0B6E1AA2EBB2E0895CF93DF9315
:1062E000C0914401CA1728F0C0914501CB1708F0AE
:1062F00003C0DF91CF910895AF93BF934F935F9306
:10630000C0913E01C53021F0C37031F0C23008F4B5
:1063100041C009F464C081C051E0AC3360F5BE32C5
:1063200050F5B0FD550FB0FD550FA0FD550FB695BA
:10633000A695CEE1BC9FD1E0C8ECCA0FD21DC00D1E
:10634000D11DA2EBB2E0CA0FDB1FA881B0912C01D6
:10635000BE70B295A07EBA17A9F0B0912C01BE70A4
:10636000AB2BAE7EA883A2EBB2E0CA1BDB0BB881DD
:10637000B52BBF70B8835F914F91BF91AF91DF9103
:10638000CF910895A2EBB2E0CA1BDB0BB881509508
:10639000B523EFCFCA2FC770C39540E00894441FC0
:1063A000CA95E9F7A695A695A695C5E1D0913E01B7
:1063B000D2FDC0E1BC9FD1E0C8ECCA0FD21DC00D18
:1063C000D11DA0912C01A695A17029F44095A8811A
:1063D000A423A883D0CFA881A42BA883CCCFCA2F75
:1063E00050912C015695537043E0C37031F0440F27
:1063F000440F550F550FCA95C9F74095A695A69518
:10640000CEE1BC9FD1E0C8ECCA0FD21DC00DD11D9A
:10641000A881A423A52BA883AECFCA2F50912C010D
:106420005E704EE0C17011F4429552954095A6956C
:10643000CAE2BC9FD1E0C8ECCA0FD21DC00DD11D6D
:10644000A881A423A52BA88396CFCE3108F0CDE157
:10645000EE3108F0EDE1D73108F0D6E1F73108F080
:10646000F6E1EC1718F40E2EEC2FC02DFD1718F4E2
:106470000F2EFD2FD02D0895EC1718F40E2EEC2FB3
:10648000C02DFD1718F40F2EFD2FD02D0895AF93BA
:10649000BF93CF93DF93EF93FF935F93D6DFAC2F40
:1064A000BD2FCF93DF93C3D1288252EBC50F52E0AB
:1064B000D51F50912C015883DF91CF91AE1711F069
:1064C000A395EFCFBF1719F0AC2FB395EACF5F912B
:1064D000FF91EF91DF91CF91BF91AF910895AF936D
:1064E000BF93CF93DF93EF93FF935F93C5DFAC2F01
:1064F000BD2FF4DEA395AE17E1F7F0DEB395FB17E1
:10650000E1F7ECDEAA95AC17E1F7E8DEBA95BD1726
:10651000E1F75F91FF91EF91DF91CF91BF91AF9143
:106520000895AF93BF93CF93DF93EF93FF935F9360
:10653000A3DFBD2FAC2FD2DEAE1711F0A395FBCF9A
:10654000CDDEFB1711F0B395F5CF5F91FF91EF9181
:10655000DF91CF91BF91AF91089599DFAF93BF9332
:10656000CF93DF93EF93FF934F935F936EDF4C2FA7
:10657000BD2FAC2F5CD152EF599351EFA395AE17BD
:1065800011F05993FBCF53EF5993A42FB395BF1735
:1065900039F04DD150EF5993AE2F49D15993F5CFE2
:1065A000A42F45D154EF599351EFA395AE1711F095
:1065B0005993FBCF55EF59935F914F91FF91EF9115
:1065C000DF91CF91BF91AF910895C7DF5F93AF93F4
:1065D000BF93CF93DF93EF93FF9337DFBD2FAC2FA4
:1065E00026D15BEF59935CEEA395AE1711F059934A
:1065F000FBCF5CEF5993FF91EF91DF91CF91CF9358
:10660000DF93EF93FF93BD2FAC2FB39510D15DEFC8
:10661000599350E2A395AE1711F05993FBCF5EEF5B
:106620005993FF91EF91DF91CF91CF93DF93EF9348
:10663000FF93BD2FAC2FB395AF93F9D0A2EBB2E08F
:10664000CA0FDB1F50912C0152955E7E2196AF91AF
:10665000A395AE1711F05993FBCFFF91EF91DF9106
:10666000CF91CF93DF93EF93FF93BD2FAC2FBE5FFE
:10667000DED05EEE59935DEEA395AE1711F05993FF
:10668000FBCF5FEE5993FF91EF91DF91CF91BF91D7
:10669000AF915F9108950F931F932F933F93AF9303
:1066A000BF93CF93DF93DE010FEFCE1B10F4019564
:1066B000C1951FEFDF1B10F41195D195CD1760F038
:1066C00000C02C2F26950ADEAE1789F0A00F2D1BD7
:1066D000D0F7B10F2C0FF7CF2D2F2695FFDDBF1769
:1066E00031F0B10F2C1BD0F7A00F2D0FF7CFDF919A
:1066F000CF91BF91AF913F912F911F910F9108952D
:10670000AF93A82DA73EE9F3A82DA73EE9F7AF91D7
:106710000895EF93FF93AF93A0931D01FBE8A6FDAF
:10672000FCE8F0932F01AF73AA0FFDE8E0E8EA0F51
:10673000F21DA591A0931A01A591A0931B0120928F
:106740001C012092180120921901AF91FF91EF9145
:10675000089520921701409117014030E1F399C04C
:10676000409116014030E1F708955FD0A2EBCA0FC7
:10677000A2E0DA1FA881BA2FAF93A171BE7EB295B5
:10678000BA2BAF912092170140911701403041F48C
:10679000409110014B3110F4A883F6CFB883F4CFA9
:1067A000A88377D042C03F933DED52D0209217018D
:1067B000409114014470431749F0403021F40E9485
:1067C0004007342F03C00E946607342F4091170101
:1067D000403061F4409110014B3120F448814F77F3
:1067E0004883E6CF488140684883E2CF58815F778D
:1067F00058833F910895D1E0C3EDCA0FD21D209276
:10680000170140911701403061F4409110014B3164
:1068100020F448814F774883F4CF4881406848830B
:10682000F0CF58815F7758830895AA2DBB2DDEE104
:10683000BD9FD1E0C8ECCA0FD21DC00DD11D089577
:10684000F6DF0F9302EBC00F02E0D01F0F91089507
:10685000D3E2BD9FD2E0C4E3CA0FD21DC00DD11D4B
:106860000895AA2DBB2DAA95B39525CDBF93BFEF53
:10687000B1B900001A99FECF42B9B4E6BA95F1F762
:106880002998B4E6BA95F1F7299ABF9108954F91E6
:1068900008954F9340912D0141FFF9CF4D7F4093D3
:1068A0002D01FF93EF93DF93CF9340913E01403052
:1068B00029F44091290147FF13C02DC04F9347E4AD
:1068C000D7D04F914F93405DD3D04F91413009F4D1
:1068D00055C0423009F469C0433009F483C093C005
:1068E00044E50E9438350E942C35C8ECD1E0FEE228
:1068F000EEE148814295A1D049919FD0EA95C9F730
:106900000E942C35FA95A1F7CF91DF91EF91FF917D
:106910004F914427089545E40E9438354091400145
:1069200089D00E942C35C8ECD1E0F3E0E3E2488145
:10693000429583D0499181D0EA95C9F70E942C35C0
:10694000FA95A1F7E3E2F0912E01EF9FC00DD11D62
:10695000F0E1E3E248814F7742956FD049914F775C
:106960006CD0EA95B9F70E942C35FA9591F7CF9142
:10697000DF91EF91FF914F914427089540910001DD
:1069800059D04091010156D067D0C8ECD1E0F4E76E
:10699000E5E14881429551D049914FD0EA95C9F738
:1069A0000E942C35FA95A1F7E2CF4091000142D028
:1069B000409101013FD0409102013CD04091030140
:1069C00039D04AD0C8ECD1E0F4E5EEE148814295F7
:1069D00034D0499132D0EA95C9F70E942C35FA9506
:1069E000A1F7C5CF39D0C8ECD1E0FAE3EAE248819B
:1069F000429523D0499121D0EA95C9F70E942C35C0
:106A0000FA95A1F7B4CF4091000114D04091010153
:106A100011D022D0C8ECD1E0F0E4E0E14881429509
:106A20000CD049910AD0EA95C9F70E942C35FA9505
:106A3000A1F79DCF4295469547704F70405D4A3310
:106A400008F0495F0C943835BF93B2E0A03009F0EC
:106A5000B064B4BDBF910895BF934F934DE0B09122
:106A60000C01B4FF05D04AE003D04F91BF910895C7
:106A7000BF93B0912501B030E1F740932601BA955C
:106A8000B0932501BF910895BF93B0912701B03015
:106A9000E1F7BA95B0932701B0912701B030E1F743
:106AA00040912801BF910895BF93B0912701B03064
:106AB000E1F7BA95B0932701409116014D3E41F0A0
:106AC000B0912701B030C1F740912801BF910895DE
:106AD0004BE1BF910895DF93CF93BF93AF93FF93A3
:106AE000EF93CEE0D7E0EEE5FBE633D0EF91FF91F8
:106AF000FF93EF93CEDECCE5D4E0B0911401B2FD6C
:106B00007E9616F026D001C01ED040911601A1E05D
:106B10004D3E69F0A2E0413F51F0A3E0423F39F021
:106B2000A4E0433F21F0A5E0443F09F0DFCFB0915E
:106B30001401B2FDAB5F4A2FEF91FF91AF91BF916E
:106B4000CF91DF910895BEE1A191A993BA95E1F7A4
:106B50000895BEE1A591A993BA95E1F708954E4E27
:106B60004E4E4E4EC0C0C0C0C0C08080808080806D
:106B70002E2E2E2E2E2E6E6E6E6E6E6EDF93CF9399
:106B8000BF93AF93FF93EF93CEE0D7E0EEE5FBE644
:106B9000E0DFEF91FF91FF93EF93CCE5D4E0D9DFF5
:106BA000CBCFACE5B0910C01B3FDAFE5ACBDACE52E
:106BB000A093B800A0E0B2FDA1E0A093B9000895B1
:106BC000FF93EF930F93E0911E01A0911F01B091ED
:106BD0002001F09121010027E2FD0095E5FD0095DF
:106BE000A4FD0095F7FD0095001FEE1FAA1FBB1F17
:106BF000FF1FE0931E01A0931F01B0932001F093AB
:106C000021010F91EF91FF910895FF93EF93DF938F
:106C1000CF93BF93AF934F935F936F937F934F92B5
:106C20005F926F927F922F9320913E014090460198
:106C3000509049016090480170904B01509147017C
:106C400060914A01A22FA370E52F660FEE0FA330CB
:106C500031F0660FEE0FA23011F0660FEE0FF62F37
:106C6000A0914C01A13071F4E20147D0803011F0C5
:106C70008FE133C0E30141D0803011F080E22DC0BC
:106C800065D02BC0A23091F4E20137D0803011F0F2
:106C90008FE123C0E30140D0803011F082E11DC0BC
:106CA000ACE3BDE06A0E7B1E75D017C0A33011F0B7
:106CB00085E113C0A52DA33010F082E10EC0ACE336
:106CC000BDE04A0E5B1EF20151916191E30115D0C6
:106CD000803011F080E201C067D02F917F906F90DB
:106CE0005F904F907F916F915F914F91AF91BF9166
:106CF000CF91DF91EF91FF910895CE0F10F48FE1C6
:106D00000895A0914401CA17D0F7DF0FC0F3B091E6
:106D10004501DB17A0F70895659FC00DD11D229690
:106D2000D33008F082E10895A22F5091470160917D
:106D30004A01E52F660FEE0FA33031F0660FEE0F1C
:106D4000A23011F0660FEE0FF62F0895571478F069
:106D5000D20134D0E0E8FBE064D0D3012FD0E0E8EA
:106D6000FBE08CD0539473946A9591F70895560E76
:106D7000760E5A947A94D20121D0E0E8FBE051D00B
:106D8000D3011CD0E0E8FBE079D05A947A946A955C
:106D900091F70895F30151936193D2010FD041D03F
:106DA00053946A95D1F70895F20151916191D301FD
:106DB00005D064D073946A95D1F708956F93C8ECA9
:106DC000D1E0213011F465E103C0253069F460E1C0
:106DD000B69FC00DD11D6A2F669566956695C60F44
:106DE000D21D4A2F6F910895223069F46EE1B69F4B
:106DF000C00DD11D6A2F66956695C60FD21D4A2F0C
:106E0000440F6F9108956AE2B69FC00DD11D6A2F9D
:106E100066956695C60FD21D4A2F440F440F6F9199
:106E200008957F936F93BF93AF93652F742F7770FF
:106E300049F4A991A1936A95E1F7AF91BF916F9140
:106E40007F910895B0E8713019F0B6957A95FBCF2F
:106E50007727A991AB9F703019F0A291A029A19337
:106E6000119273957617A9F7A991AB9FA291A029CA
:106E7000A193AF91BF916F917F9108957F936F938D
:106E8000BF93AF93652F742F777049F4A191A993A5
:106E90006A95E1F7AF91BF916F917F9108950F933C
:106EA0001F930FEF11E0000F110F7A95E1F7652F97
:106EB0007881009570230095A191A19F072A0992DE
:106EC000712D6A95C9F768816023672B69930F91CB
:106ED0001F91AF91BF916F917F910895BF93AF9331
:106EE0004F939927A42F0E94332F0E94B32F4F91C5
:106EF000AF91BF910895AF93BF93EF93FF935F93CB
:106F00006F930F931F932F9310E020E0FAE8EE2782
:106F1000509147015F7760914A016F770491059F17
:106F2000A12DE0950491E095069FB12DA11729F4BC
:106F3000B21719F4E39591F724C01A2F2B2FA091C3
:106F40004601B0914901A10FB20F0E946E31A0918C
:106F50004601B0914901A10FB21B0E946E31A09170
:106F60004601B0914901A11BB21B0E946E31A09154
:106F70004601B0914901A11BB20F0E946E31E39509
:106F800069F62F911F910F916F915F91FF91EF9192
:106F9000DF91AF910895AF93BF93EF93FF935F930A
:106FA0006F930F931F932F933F932FEFFAE8EE27E2
:106FB000509147015F7760914A016F770491059F77
:106FC000A12DE0950491E095069FB12DB21721F413
:106FD000E395A1F73F91D5CF1A2F2B2FA091460112
:106FE000B09149013A2FB21BA11B310F0E946E31A3
:106FF000B20FB20F0E946E31B21BB21BA3953A17AB
:10700000A8F7E395D9F63F91BCCFFF91EF91EE0F32
:10701000FF1F5BD03197F695E7953196EF93FF937D
:10702000C8E7D1E040912C014F93FF93EF9361D0DB
:107030000E9442310B0920505245535320454E5473
:1070400045522000EF91FF914F9140932C0181DB3D
:107050004A3EE9F785DB0E941A1A0895FF91EF91E5
:10706000EE0FFF1F32D03197F695E7953196EF93EB
:10707000FF93C8E7D1E040912C014F93FF93EF932A
:1070800038D00E9442310B08202859296573202FDF
:1070900020284E296F200000EF91FF914F914093DF
:1070A0002C0157DB493761F0493551F04E3619F064
:1070B0004E3409F0F6CF54DB0E941A1A4427089583
:1070C0004FDB0E941A1A41E00895C8E7D1E04591CC
:1070D00046954F93477049934F9142954770499316
:1070E00058E145914993403011F05A95D1F72992D2
:1070F0000895FF93EF9392E020922A01A991B9910C
:10710000B295B077A770AB0FAA0FA0932C01DF93B5
:10711000CF930E94F419C2E0D8E0EBE1FCE00E94BA
:10712000AD32A3E0B9E00E945B31CF91DF9158E12D
:107130004991403051F0DF93CF935F930E94B42F79
:107140005F91CF91DF915A9599F740912C0142952B
:1071500040932C01EF91FF910895FF93EF93DF93FC
:10716000CF93BF93AF93C0914601D09149010A815B
:1071700019810E3118F4173108F41AD0A091480182
:10718000B0914B01C0914601D0914901B983AA83C6
:10719000AE3138F4B73128F43DD07370713009F056
:1071A00076D0AF91BF91CF91DF91EF91FF9108958C
:1071B000C0914601D09149010A8119812C813B81FE
:1071C000239F310F2596C00DD11DC00DD11D412F1C
:1071D000E8ECF1E05EE1549FE00DF11DE00FF21DDF
:1071E000522F699161935A95E1F74395431781F7BF
:1071F000412FEAE7F4E05EE1549FE00DF11DE00F5E
:10720000F21D522F699161935A95E1F74395431707
:1072100081F70895C0914601D09149010A811981F1
:107220002C813B81239F310F2596C00DD11DC00DB0
:10723000D11D7727412FE8ECF1E05EE1549FE00D8E
:10724000F11DE00FF21D522F619169936F7009F0EB
:1072500071E05A95C9F74395431769F7E0914601E4
:10726000F09149014081742B7083412FEAE7F4E0EB
:107270005EE1549FE00DF11DE00FF21D522F619170
:1072800069935A95E1F74395431781F70895C091A3
:107290004601D09149010A8119812C813B81310F2E
:1072A0002596412FE8ECF1E05EE1549FE00DF11DE1
:1072B000E00FF21D522F699161935A95E1F74395C2
:1072C000431781F7412FEAE7F4E05EE1549FE00DB8
:1072D000F11DE00FF21D522F6991660F28F46E70B8
:1072E000462E6081607F642961935A95A9F7439582
:1072F000431749F70895AF93BF93CF93DF934F930D
:107300005F936F937F934F9270912C014370E1F4E0
:10731000A6E0B2E0C4E2D2E0422C07D0A8EBB4E091
:10732000C6EDD4E0472E01D061C062E15AE1499137
:107330004D935A95E1F7149624966A95B9F75AE158
:107340004D925A95E9F708954130C9F4ACE3B4E0A1
:10735000CBE3D4E0422C07D0AEEEB6E0CDEED6E0E3
:10736000472E01D043C063E159E14A914E935A95AB
:10737000E1F74E92149725976A95B1F70895423038
:10738000E1F4ACE3B4E0CEE1D4E0422C07D0AEEEC1
:10739000B6E0C0EDD6E0472E01D028C062E15AE148
:1073A0004A914E935A95E1F7149724976A95B9F745
:1073B0005AE14E925A95E9F70895A6E0B2E0C7E087
:1073C000D2E0422C07D0A8EBB4E0C9EBD4E0472EC2
:1073D00001D00CC063E159E149914D935A95E1F711
:1073E0004D92259614966A95B1F708954F907F9126
:1073F0006F915F914F91DF91CF91BF91AF910895C0
:107400004F935F937F9350DB4B3111F481E015C0B4
:107410004130C9F739DB642F37DB4095641711F031
:1074200088E20BC070E855272FDB540F49937A95FB
:10743000D9F72ADB451729F488277F915F914F916F
:10744000089589E2FACF4F935F937F9341E010DB79
:10745000462F0EDB40950CDB70E855274991540F01
:1074600007DB7A95D9F7452F03DB7F915F914F9129
:1074700008955E984CE54093B80044E84093BC0002
:1074800044E94093BC00089544EA0EC05093BB0009
:1074900044E80AC044EC08D05091BB00089544E889
:1074A00003D05091BB0008954093BC004091BC00B4
:1074B00047FFFCCF6091B900687F0895E5DF683031
:1074C00089F4572F550F5E70506AE0DF683151F430
:1074D0005B2FDCDF683231F45A2FD8DF683211F4C9
:1074E000882708958FE05F915F91CACFE7DFCCDFF7
:1074F000603169F4572F550F5E70516AC7DF6034F1
:1075000031F4CDDF683519F411968827B9CF8FE0B3
:10751000B7CF052ED3DF502DB9DF683219F411969D
:107520008827AECF8FE00895AFDF6830A9F4572FDA
:107530005770550F5169AADF603471F4ABDF6035C5
:1075400059F4A52FACDF683539F4BB27550FAA1FB6
:1075500008F4B095882794CF8FE092CF8827D83051
:1075600020F080E34F914F914FEF0895F7DFF999A5
:10757000FECFD2BDC1BDF89A40B521960895EEDF89
:10758000F999FECFD2BDC1BDF89A40B4441611F4AA
:107590002196089554E040BDF894FA9AF99A7894A7
:1075A000F999FECFF89A40B4441511F42196089544
:1075B000839580635A9579F70895AF93D7DF419308
:1075C000AA95E1F7AF910895AF934191D8DFAA95BD
:1075D000E1F7AF9108954EBD4DB547FFFDCF4EB5D4
:1075E000089588272C9847EDF6DF4427F4DF2C9A7E
:1075F0004C7B4432B1F34C31A1F38827443A19F063
:107600004C3909F081E108958827EBDF803021F0C3
:1076100040E040939C1008954C3911F448E0F9CFB4
:1076200040E1F7CFF1DF403009F40895440F440FF3
:10763000440F440F4A950895AA0FBB1F4B2FCBDF71
:107640004A2FC9DF422DC7DFB695A7950895803030
:1076500059F44F93C6DF803031F42C9845E5BBDFF9
:10766000EBDF2C9ABEDF4F910895803059F44F9391
:10767000B8DF803031F42C9843E5ADDFDDDF2C9AA4
:10768000B0DF4F910895803051F44F93AADF8030DE
:1076900029F42C9846E89FDFCFDF2C9A4F9108956C
:1076A0001196B0939D10A0939E101197ECCF7F93ED
:1076B000772710D07F9108957F9371E00BD0D42F5E
:1076C00072E008D0C42F7F9108957F9373E002D0B9
:1076D0007F9108958030B9F484DF8030A1F42C9834
:1076E00042ED79DFAA0FBB1FA3954B2F74DF4A2F02
:1076F00072DF472F70DFB695A7956DDF6CDF6BDF0C
:107700006ADF69DF2C9A08958030D1F46ADF803017
:10771000B9F42C9842ED5FDFAA0FBB1F4B2F5BDF44
:107720004A2F59DF472F440F56DFB695A79553DFF1
:1077300052DF51DF50DF4FDFD42F4DDFC42F2C9AA3
:1077400008957F9370E010D07F9108957F9371E04A
:107750004D2F0AD072E04C2FBDDF7F9108957F93AB
:1077600073E0B8DF7F9108958030A1F44F9339DF43
:107770004F91803079F42C984F9347E82CDF4427C1
:107780002ADF41E028DF472F26DF4F914F9323DF89
:107790002C9A4F910895803091F423DF8030D1F7F7
:1077A0002C984F9347E817DF442715DF40E013DF9D
:1077B000472F11DF4F914F930EDF2C9A4F91089571
:1077C0008030D1F4DF93CF934F935F930ADF803003
:1077D00079F42C9847E8FFDE4427FDDE4427FBDEE2
:1077E00040E0F9DE55274991F6DE5A95E1F72C9AEB
:1077F0005F914F91CF91DF9108958030B1F44F9315
:107800005F93EFDE803079F42C9847E8E4DE44277C
:10781000E2DE4427E0DE40E0DEDE55274FEFDBDE30
:107820005A95E1F72C9A5F914F9108958030E1F4D9
:10783000DF93CF934F935F93D4DE803089F42C98FD
:1078400046EDC9DE4427C7DE4427C5DE40E0C3DE7F
:107850004427C1DE5527BFDE49935A95E1F72C9A9C
:107860005F914F91CF91DF910895BF93AF93DF93D5
:10787000CF934F935F937F93C7DE403041F47F9166
:107880005F914F91CF91DF91AF91BF910895B5DF97
:107890004FE057DF442763DFAA27BB27F4DE1196AA
:1078A0004DEFCA2FCF70C13009F44CEF4ADF4427A7
:1078B00056DFCC27DD274ADFE6DE1196A03019F42B
:1078C00045EE0E94B42F40919C10B41749F7D7CFD2
:1078D000BF93AF93DF93CF934F935F937F9394DEE8
:1078E000403091F47F915F914F91CF91DF91AF91B3
:1078F000BF910895B42FAA271197E7DEC42FBB27A5
:10790000AA27E3DE4C1731F4A2DEDFDE439527DF42
:10791000BADEE8CF1196D9DE4C17E1F7F5CFDF9349
:10792000CF934F9394DE4DEFCA2FCF70C13009F43F
:107930004CEF07DFC1DE219609DF5FDFA4DE4F9148
:10794000CF91DF910895FF93DF93CF93BF93AF93D0
:10795000AA27BB27ED0158DE4030A1F0F42FA7DEA7
:107960004C3F41F04D3F31F04B3A21F04F3018F091
:10797000403908F421961196BF1789F74427DF177D
:1079800009F441E0AF91BF91CF91DF91FF9108954C
:107990000F93BF93AF934F93AA27BB27ED01FD0130
:1079A00033DE403099F0042F82DE4D3F49F4DF93FF
:1079B000CF9382DE4D2FCF91DF914F3F21F0219663
:1079C0004C3F09F431961196B01771F74F91AF9172
:1079D000BF910F910895FF93EF93DF93CF934F9350
:1079E0002F9312DE4030A9F0AA27BB2760DE242F98
:1079F000B0919D10A0919E1040910801B41710F015
:107A0000A2E0BB27FD0153DE4D3F51F455DED217F6
:107A100038F42F914F91CF91DF91EF91FF9108951D
:107A2000159640919C10B41709F4BB27BF1759F75E
:107A3000AE1749F7AA27BB270ADE39DE4F3F31F0E0
:107A4000405F242F7EDE1FDEDF01DDCFAFEFBFEF13
:107A5000E0CFFF93EF93DF93CF93BF93AF934F9319
:107A60005F936F937F93D0DD403061F481E17F912C
:107A70006F915F914F91AF91BF91CF91DF91EF9156
:107A8000FF91089551D0B41710F08BE1F0CF0FDEC5
:107A90004C3F11F087E1EBCF40915A01403011F497
:107AA0008BE1E5CF413810F08BE1E1CF71DFD030D1
:107AB00021F4C41710F488E1DACFC0E8DBE050E02D
:107AC0006FEF69935A95E9F798DE1196B0939D1080
:107AD000A0939E1040915A01C0E8DBE04F937BDFFA
:107AE000B993A9934BEA2DDEDF93CF93E5DD219681
:107AF0002DDECF91DF91E9DD32DED2DDE9DE4F917F
:107B00004A9561F711D0C0E8DBE05ADE40915C0194
:107B100018DEDF93CF93D0DD219618DECF91DF9171
:107B2000D4DD1DDEB0DDA3CFA0915801A295BA2F00
:107B3000A07FBF7011960895BF93AF93DF93CF934B
:107B40004F935F937F937727EFDFB1DD4C3F69F071
:107B5000DBDDDF3F49F0BF93AF93DE01E0DEAF91A5
:107B6000BF91B6DE7F5FA1F7DADE7F915F914F9123
:107B7000CF91DF91AF91BF910895BF93AF93DF9302
:107B8000CF934F935F937F932F93AA27BB2729DD32
:107B90008EDD242FC9DF8BDD4C3F51F489E12F911D
:107BA0007F915F914F91CF91DF91AF91BF910895F8
:107BB00070915A01703810F08BE1F1CFA5DDDF3FF5
:107BC00011F48BE1ECCFDE01CCE3DDE040915C0110
:107BD000413009F4D395423009F4DE5FF1DDDF93E3
:107BE000CF936ADDD21759F02196B0DDCF91DF91A6
:107BF0005EDDA7DD6ADDB3DD46DD6ADED0CF8FDE78
:107C0000EADE5ADD2196A2DDCF91DF914BEA99DDC4
:107C10005CDDA5DD38DDED0187DF19DD70915A01EE
:107C2000770F4D2FB8DD73954C2FB5DD40DD89DD25
:107C30004CDD95DD28DDB3CFBF93AF93DF93CF93BA
:107C40004F935F937F9370DF32DD4C3F49F48EE1B9
:107C50007F915F914F91CF91DF91AF91BF91089547
:107C600070915A01703810F08BE1F2CF4DDDDF3F9B
:107C700011F48BE1EDCFDE01EADCCCE3DDE04091F5
:107C80005C01413009F4D395423009F4DE5FCEDD6A
:107C9000DFCF0004080D11161A1F23282C303539A8
:107CA0003D42464A4F53575B5F64686C7074787C02
:107CB0007F83878B8F92969A9DA1A4A7ABAEB1B517
:107CC000B8BBBEC1C4C6C9CCCFD1D4D6D9DBDDDFE9
:107CD000E2E4E6E8E9EBEDEEF0F2F3F4F6F7F8F9BA
:107CE000FAFBFCFCFDFEFEFFFFFFFFFFFFFF0000B5
:107CF00000CCC000333000FFF000000CCCCCCCCC6A
:107D0000333CCCFFFCCC000333CCC333333333FFE1
:107D1000F333000FFFCCCFFF333FFFFFFFFFA5A5DD
:107D2000A506FF6000000000000000000000000049
:107D30000000000000000000000000000000000043
:107D400000000EAE000004E000AAE800EE4E0000C5
:107D500000444040AA000066FF666842C4A248A0F2
:107D60000000004400004888404222400A4A0004C3
:107D7000E40000048000E000000040224880EAAAFD
:107D8000E04C44E0E2E8E0E2E2E0AAE220E8E2E0FF
:107D9000E8EAE0E24880EAEAE0EAE2E0040400041B
:107DA00004802484200E0E00842480C268E400EE47
:107DB000E04AAEA0CACAC0688860CAAAC0E8C8E0E3
:107DC000E8C88068EA60AAEAA0E444E0E22A60AC7D
:107DD0008CA08888E0AEAAA0CAAAA04AAA40EAE875
:107DE000804AAA60EAECA068E2C0E44440AAAAE0A3
:107DF000AAAA40AAAEA0AA4AA0AA4440E248E064C7
:107E0000446004A400C444C04A00000000E04400F0
:107E1000004AAEA0CACAC0688860CAAAC0E8C8E062
:107E2000E8C88068EA60AAEAA0E444E0E22A60AC1C
:107E30008CA08888E0AEAAA0CAAAA04AAA40EAE814
:107E4000804AAA60EAECA068E2C0E44440AAAAE042
:107E5000AAAA40AAAEA0AA4AA0AA4440E248E024A6
:0E7E6000C4204444448464808842208CEC801A
:1086000000F900F5F3F1F2FC00FAF8F6F4EB5E0085
:10861000F7000000007131000000797361773200CB
:108620000063786465343300002076667472350028
:10863000006E6268677A360000006D6A7537380030
:10864000002C6B696F303900002E2D6C00707E009D
:1086500000000000002700000000EA2B00230000BB
:10866000003C00000000EC00003100343700000046
:10867000302C32353638ED00FB2B332D2A390000F3
:1086800000F900F5F3F1F2FC00FAF8F6F4EB000063
:10869000F70000000051210000005953415722000B
:1086A00000435844452440000020564654522500BB
:1086B000004E4248475A260000004D4A552F2800D8
:1086C000003B4B494F3D2900003A5F4C00503F00B2
:1086D00000000000006000000000EA2A00270000FF
:1086E000003E00000000EC000031003437000000C4
:1086F00030E932353638ED00FB2B332D2A390000B6
:108700000000000000000000000000000000000069
:108710000000000000000000000000000000000059
:108720000000000000000000000000000000000049
:1087300000000000000000C000000000000000C1B8
:10874000000000000000000000002F0000000000FA
:1087500000000000000000000000EA000000C2006D
:10876000000000000000000000E100E2E000000066
:10877000E8E9E500E3E4ED00FB2BE72D2AE6000045
:1087800000000000000000000000000000000000E9
:108790000000000000400000000000000000000099
:1087A00000000000000000000000000000000000C9
:1087B000000000000000000000000000007B5B00E3
:1087C00000000000007D5D000000000000007E0051
:1087D00000000000000000000000005C000000003D
:1087E000007C00000000000000E100E2E00000006A
:1087F000EFEEE500E3E4ED00FB2BE72D2AE60000B9
:1088000000F900F5F3F1F2FC00FAF8F6F4EB5E0083
:10881000F70000000071310000007A7361773200C8
:108820000063786465343300002076667472350026
:10883000006E62686779360000006D6A753738002F
:10884000002C6B696F303900002E2F6C3B702D00AF
:10885000000027005B3D00000000EA5D007E000094
:10886000000000000000EC00003100343700000080
:10887000302C32353638ED00FB2B332D2A390000F1
:1088800000F900F5F3F1F2FC00FAF8F6F4EB000061
:10889000F70000000051210000005A5341574000EA
:1088A00000435844452423000020564654522500D6
:1088B000004E424847595E0000004D4A55262A00A6
:1088C000003C4B494F292800003E3F4C3A505F0086
:1088D000000022007B2B00000000EA7D007C0000ED
:1088E000000000000000EC00003100343700000000
:1088F00030E932353638ED00FB2B332D2A390000B4
:108900000000000000000000000000000000000067
:108910000000000000000000000000000000000057
:108920000000000000000000000000000000000047
:1089300000000000000000C000000000000000C1B6
:10894000000000000000000000002F0000000000F8
:1089500000000000000000000000EA000000C2006B
:10896000000000000000000000E100E2E000000064
:10897000E8E9E500E3E4ED00FB2BE72D2AE6000043
:1089800000000000000000000000000000000000E7
:1089900000000000000000000000000000000000D7
:1089A00000000000000000000000000000000000C7
:1089B00000000000000000000000000000000000B7
:1089C00000000000000000000000000000000000A7
:1089D0000000000000000000000000000000000097
:1089E000000000000000000000E100E2E0000000E4
:1089F000EFEEE500E3E4ED00FB2BE72D2AE60000B7
:108A0000FFFFFFFFFFFFFFFFFFFFFFFEFEFEFEFE7B
:108A1000FEFEFDFDFDFDFDFCFCFCFCFBFBFBFBFA93
:108A2000FAFAF9F9F9F8F8F8F7F7F6F6F6F5F5F4D1
:108A3000F4F3F3F2F2F2F1F0F0EFEFEEEEEDEDEC35
:108A4000EBEBEAEAE9E8E8E7E6E6E5E4E4E3E2E1BD
:108A5000E1E0DFDEDEDDDCDBDADAD9D8D7D6D5D46B
:108A6000D4D3D2D1D0CFCECDCCCBCAC9C9C8C7C63A
:108A7000C5C4C3C2C1BFBEBDBCBBBAB9B8B7B6B529
:108A8000B4B2B1B0AFAEADACAAA9A8A7A6A5A3A237
:108A9000A1A09E9D9C9B99989796949392918F8E5E
:108AA0008D8B8A898786858382817F7E7D7B7A789C
:108AB0007776747371706F6D6C6A696766656362EF
:108AC000605F5D5C5A595756545351504E4D4B4A56
:108AD0004847454442413F3E3C3B393836353332C6
:108AE000302E2D2B2A2827252422201F1D1C1A1941
:108AF00017161412110F0E0C0B09070604030100C0
:108B00000C11161A1E2225282B2D2F313233333407
:108B100034343434343434343535363738393B3CF6
:108B20003E40434547494B4D4F5152535454545482
:108B3000545351504E4C4A4745423F3D3A383634E3
:108B40003231302F2E2E2E2F303132333536383A07
:108B50003C3E4042444647494A4B4D4E4E4F505092
:108B60005050505050504F4E4D4C4B494846434149
:108B70003E3B37332F2B27221D18130D0802FDF81B
:108B8000F3EEE9E5E1DDDAD7D4D2D0CECDCCCCCB53
:108B9000CBCBCBCBCBCBCBCBCACAC9C8C7C6C4C344
:108BA000C1BFBCBAB8B6B4B2B0AEADACABABABAB98
:108BB000ABACAEAFB1B3B5B8BABDC0C2C5C7C9CB17
:108BC000CDCECFD0D1D1D1D0CFCECDCCCAC9C7C5D3
:108BD000C3C1BFBDBBB9B8B6B5B4B2B1B1B0AFAF28
:108BE000AFAFAFAFAFAFB0B1B2B3B4B6B7B9BCBE51
:108BF000C1C4C8CCD0D4D8DDE2E7ECF2F7FD02075F
:108C0000000A141D272F383F464B505457595959C5
:108C1000585654504C48433E39332E2925201C19B0
:108C200016141211111112131517191C1F222527C2
:108C30002A2C2E303132323232312F2D2B28252260
:108C40001F1C191613110F0D0C0B0A0A0A0B0C0E20
:108C500010121416181A1C1E1F2020201F1E1C196B
:108C600016120D0803FDF7F0EAE3DDD6D1CBC6C23C
:108C7000BFBDBBBABBBCBEC2C6CBD1D7DFE6EFF728
:108C80000008101920282E34393D41434445444200
:108C9000403D39342E29221C150F0802FCF7F2ED55
:108CA000E9E6E3E1E0DFDFDFE0E1E3E5E7E9EBED83
:108CB000EFF1F3F4F5F5F5F4F3F2F0EEECE9E6E3B9
:108CC000E0DDDAD7D4D2D0CECDCDCDCDCECFD1D37D
:108CD000D5D8DADDE0E3E6E8EAECEDEEEEEEEDEB3A
:108CE000E9E6E3DFDAD6D1CCC6C1BCB7B3AFABA9F6
:108CF000A7A6A6A6A8ABAFB4B9C0C7D0D8E2EBF57B
:108D000080675342352B221C16120E0C09070605EC
:108D1000040000000000000000000000000000004F
:108D20000000000000000000000000000000000043
:108D30000000000000000000000000000000000033
:108D40000000000000000000000000000000000023
:108D50000000000000000000000000000000000013
:108D60000000000000000000000000000000000003
:108D700000000000000000000000000000000000F3
:108D8000890091009A00A300AD00B700C200CE0098
:108D9000DA00E700F4000301120123013401460167
:108DA0005A016E0184019B01B301CD01E901060264
:108DB0002502450268028C02B302DC020803360376
:108DC00067039B03D2030C0449048B04D0041905E8
:108DD0006705B90510066C06CE063507A307170808
:108DE000930815099F09320ACD0A720B200CD80C82
:108DF0009C0D6B0E460F2F1025112A123F13641481
:108E0000F894A0E02A2EA1E03A2EA0E1AEBFAFEF89
:108E1000ADBFB0E0A0E0AA95F1F7BA95D9F7AAEBFB
:108E2000A4B9AFEFA5B9A0E8A7B9A0E0A8B9A0EF91
:108E3000AAB9AFEFABB9A6B1AF71A09329014B9915
:108E40005DC0B2ECB0938000B9E1B0938100F4E072
:108E5000A2FFF4E0F0938700FEEFA2FFF6EFF0939D
:108E6000860020928900FAE5F0938800A2E0A093A2
:108E70006F00A0E4A4BDA1E0A5BDA1E3A7BD209221
:108E8000C000A0E1A093C100A6E6A093C200E0EA62
:108E9000FFE87ED0A2E2B591B993AA95E1F705B7B4
:108EA000036005BF0E7F05BF7894A8EC68D0B09131
:108EB000C600B83719F0AA95C9F720C0E0ECFFE862
:108EC00067D045E140D0C8ECD1E020D046E03BD0AF
:108ED000E0E0F0E0CCE3DFE019D046E034D0CCEBCA
:108EE000DFE014D0FE3820F40E947A79329678942C
:108EF00046E029D0AEEDB1E01BD0ECCFF89405B739
:108F0000016005BF0C7F05BF0C94000028D04430E1
:108F100039F446E018D0B0912501B030E1F7EECF3A
:108F200050E81DD01CD01BD049935A95E1F717C0CB
:108F30004F2F429501D04F2F4F70405D4A3308F0BC
:108F4000495F4D930895BF93B0912501B030E1F78B
:108F500040932601BA95B0932501BF910895BF9320
:108F6000B0912701B030E1F7BA95B0932701B091E5
:108F70002701B030E1F740912801BF910895AF93E8
:108F8000A82DA73EE9F3A82DA73EE9F7AF910895D4
:108F9000C8ECD1E0A2E2B591B993AA95E1F70895A2
:108FA0004156522D436869704261736963322028CB
:108FB0004631313D557064617465205379732920C1
:108FC000426F6F746C6F61646572204572726F726C
:108FD000202845534320746F206578697429202028
:0E900000202020202020202020202020FFFFE4
:0E9C0000202020202020202020202020FFFFD8
:0EA80000202020202020202020202020FFFFCC
:0EB40000202020202020202020202020FFFFC0
:0EC00000202020202020202020202020FFFFB4
:0ECC0000202020202020202020202020FFFFA8
:0ED80000202020202020202020202020FFFF9C
:0EE40000202020202020202020202020FFFF90
:10F000000C94004700000000000000000000000019
:10F0100000000000000000000000000000000000F0
:10F0200000000000000000000000000000000000E0
:10F03000000000000C941C784F935F936F93FF9334
:10F04000EF93DF93CF93BF93AF930F921F92FFB7CE
:10F05000FF93C8E0D1E0B9A5B7FF5C98B7FD5C9A13
:10F060004B99BE7F4B9BB160B9A7830C921CE9A161
:10F07000F92DF03029F4F82DFA3010F1F63EF8F0C1
:10F08000FCE0E2FFFDEE8F1639F45E98E3FF17C057
:10F09000B2E8B093800013C0F1E1E2FFF3EF8F1606
:10F0A00039F45E9AE3FF0BC0B2ECB093800007C066
:10F0B000F9E3E2FFF7E08F1611F4882499242CC0BD
:10F0C000A0918400AA3FE0F3AB3F00F0AC3F00F01A
:10F0D000AD3F00F0AE3F00F0A8ECB1E0F6EFF80D68
:10F0E000C0E2ED91549140E060E848B9ED9156FDE1
:10F0F00066B90000000055FD66B9049054FD66B97C
:10F10000CA95000053FD66B90000000052FD66B9C3
:10F11000502D59F7000028B814D0E091C600E6370A
:10F1200011F40C947E47FF91FFBF1F900F90AF9199
:10F13000BF91CF91DF91EF91FF916F915F914F91CF
:10F140001895A0913101E0912701E03091F0EF3F57
:10F1500021F4A0FD0EC0EEE30CC0EA95F5EFB491EA
:10F16000B5FF07C0B0912801B695A0FBB7F9B093E1
:10F170002801E0932701E0912501E03091F0EF3F75
:10F1800019F4E8E4AF770DC0EA95F5EFB491B4FF58
:10F1900008C0B0912601B0FB0894B795A7F9B093C9
:10F1A0002601E0932501A09331010895A09131013A
:10F1B000E0912701E03091F0EF3F21F4A0FD0EC077
:10F1C000ECE70CC0EA95F5EFB491B7FF07C0B0913A
:10F1D0002801B695A0FBB7F9B0932801E093270169
:10F1E000E0912501E030E9F2EF3F19F4E0E9AF7773
:10F1F000D8CFEA95F5EFB491B6FFD3CFB091260101
:10F20000B0FB0894B795A7F9B0932601CACF4091F7
:10F210000C01C8EFD7E00E94BF3A0895C8EFD7E0CD
:10F220000E94B63A40930C010895C9EFD7E00E94BE
:10F23000BF3A0895CF93DF93C9EFD7E00E94B63A63
:10F24000742FDF91CF910895FF93EF93DF93CF93C6
:10F25000AF93F4D0E0933401F0933501AF91CF91A7
:10F26000DF91EF91FF910895E0E0F0E9C0E0DCE08C
:10F27000A42FA03021F0EC0FFD1FAA95FACF08951E
:10F28000E0913401F0913501A0E2A99FE00DF11D5C
:10F29000B096C0EAD1E0A0E2B591B993AA95E1F7A2
:10F2A000BFEFB993089547B740FDFDCFB7BFE895CD
:10F2B00047B740FDFDCF089547B746FF0895B1E138
:10F2C000F2DFFACFF8944E2F407E19F4B3E0EBDF73
:10F2D000F3DFA0E109901990B1E0E5DF3296AA953D
:10F2E000C9F7E03009F008953297B5E0DCDFE4DFDC
:10F2F00032960895F8944F93BF93AF93B3E0D3DF62
:10F30000DBDF3297CCE3DFE0A0E83296099019907A
:10F31000B1E0C9DFAA95C9F7B5E0C5DFCDDFAF9190
:10F32000BF914F910895E0913401F0913501B0976C
:10F33000ACE0B591B993AA95E1F7A0912901A7FD99
:10F340000895A6EAB2E0CA0FDB1FACE0B0912C0131
:10F35000B993AA95E9F70895E0E0F0E9A0E0BCE0F0
:10F36000492F403029F3EA0FFB1F4A95FACFF89452
:10F3700063D0C0EAD1E0A3EDB1E05CE04D914993E8
:10F380005A95E1F742E4499353E140E2B9935A9523
:10F39000E9F7A09797DF9927B3E2B99FA4E3B2E01A
:10F3A000A00DB11DC8E7D1E050E24D9149935A95A7
:10F3B000E1F7299250E24A91403219F428825A9595
:10F3C000D1F70E945C18C0EAD1E07CDF93959F35AD
:10F3D00019F77894089530D0A3EDB1E05CE0459141
:10F3E0004D935A95E1F77496992750E2A0EAB1E05F
:10F3F00045914D935A95E1F7A8E7B1E040E253E219
:10F400004D935A95E9F7FF93EF939F930E94461906
:10F410009F91EF91FF91C8E7D1E0B3E2B99FA1E3DB
:10F42000B2E0A00DB11D53E249914D935A95E1F719
:10F4300093959F35D1F6089540913D01AF93BF93C9
:10F44000E0E0F0E947704295A0ECA49FE00DF11DCB
:10F45000BF91AF910895CCE3DFE04CE050E25993C7
:10F460004A95E9F75FEF599343E150E259934A9582
:10F47000E9F740EF5FEF59934A95E9F7DDDF3ADFAF
:10F480003296CCE3DFE040E25FEF59934A95E9F72B
:10F490004BE04F932FDF32964F914A95D1F77894F6
:10F4A0000895472F4770CADFFF93EF93C5DFAF91F1
:10F4B000BF914CE04F93CCE3DFE040E0559159938E
:10F4C0004A95E1F7FF93EF93FD0114DF3296DF01D8
:0EF4D000EF91FF914F914A9569F77894089556
:10F50000010101010101210101010101013181011B
:10F510000100003100010101010131C101010101BE
:10F520003101010101010131C1010101013101017B
:10F530000101010131C101010101110101010101BB
:10F540000111C1010101010101010101010101C11B
:10F55000010101010101010101000101C1010101DC
:10F56000010101010101010001C1010101010100CD
:10F57000010101010101410001010101010101003D
:10F58000000000400000000000000000000000003B
:10F59000000000000000000000000000000000006B
:10F5A000000000000000000000000000000000005B
:10F5B000000000000000000000000000000000004B
:10F5C000000000000000000000000000000000003B
:10F5D000000000000000000000000000000000002B
:10F5E000100000000000000000000000000000000B
:10F5F00020000000000000000000000000000000EB
:10F60000009010800090108000901080009010807A
:10F61000FC28288004C0145028282800000000007E
:10F6200000000000000000000000000000000000DA
:10F6300000000000000000000000000000000000CA
:10F6400000000000000000000000000000000000BA
:10F6500000000000000000000000000000000000AA
:10F66000000000000000000000000000000000009A
:10F67000000000000000000000000000000000008A
:10F6800028C004C00000000000000000000000804E
:10F69000C0A0888400000000000000002088FCB4A6
:10F6A0000028000008A08080000004C028800024FA
:10F6B00000008000000044288000C004C41800003E
:10F6C00004C0008004C000C400000000000000006E
:10F6D0008090808008A084408080C8A400004C8472
:10F6E000000000000000000000000000008028284A
:10F6F000280000002828002828282800002CE8904E
:10F700000090108000901080009010800090108079
:10F710007C444480A8A814504844440024000000BD
:10F7200000183C3C185028280C3000000000000055
:10F73000241824400C401440242400000C003024E1
:10F7400024244424444040246424106460646424D9
:10F7500044244424406464646464404800481800BD
:10F76000300060000400140060180C6028000000E5
:10F7700000000000300000000000000C18306000A5
:10F7800028A004C0808044283C3C3C000044A88061
:10F79000C0A08884000000000000008040847C58E5
:10F7A000182800001090808004C004C028FC287C29
:10F7B00000440C00000044EC8000C004C42400009D
:10F7C00008A000800C6000C40000000000000000E1
:10F7D0008088A41010908440C004C8A400008C80CD
:10F7E000287C008080000000000000000000244809
:10F7F000280000002828002828282800002CE8C01D
:10F800000090108000901080009010800090108078
:10F81000FC44448080801450444444283C00000050
:10F8200000183C3C20546C181818181800000004EC
:10F830006428640C14603064646428281800186418
:10F84000646464646460606464180C6C605864642C
:10F8500064646464186464646464046000183C0054
:10F860001800600004003400600000601800000010
:10F870000000000030000000000000181818601898
:10F88000449008A0C4C4806C0000001C1844A880E8
:10F89000C0A0888400000000000080804084FCB488
:10F8A0002428282820888080A4A00C60448044401C
:10F8B00000440C40844444800000C0046C24004494
:10F8C00008A000800C6000C4000000000000481088
:10F8D0008084BCB020888820D834C8A440848C8020
:10F8E0002C7C00C4C444000000000000008020887C
:10F8F000280000002828002828282800002CE8A03C
:10F900000090108000901080009010800090108077
:10F910007C808080808010908480804424186424BF
:10F9200000183C40780C7830300C7C180000000C3B
:10F93000681804183C44600C6464282830400C04A7
:10F94000046464606460606064180C78607C546473
:10F9500064646460186464643C640C60301864001F
:10F960000C2444242C2430207428146C185C742437
:10F970004824742448646464646440181818300C83
:10F9800044881090C4BC446C24246434286C6C807B
:10F99000C0A08884000000000080808080807CEC13
:10F9A000404444442088408490A00C6044FC286477
:10F9B00000440C40844444280000C0046C240080AF
:10F9C000109000441830006C00000000000018186F
:10F9D0008080BC1040848820E82CC8A480804C849F
:10F9E000EC2400C4EC4400000000000000802088EB
:10F9F000280000002828002828282800002CE8E4F7
:10FA00000090108000901080009010800090108076
:10FA1000FC808080B098109080ECEC44003C6464E2
:10FA20000018003C24183000300C2440004000181E
:10FA30007C180C0C6C044418242000006000040C9A
:10FA40002C6444606444447040180C50607C7C64B6
:10FA50004464442418646464183C18607C180000F2
:10FA6000000464606864486454180C78187C54641A
:10FA70006C6C5460306464643C640C30180C188006
:10FA800080841090C4F8806C04646440406C6C8086
:10FA9000C0A0888400000000808080808080FCB44A
:10FAA0001880442840844084808418308080282432
:10FAB00000440C40844444440000C00428241880BE
:10FAC000109000441830006C00000000000040243A
:10FAD000A4B0BC4080808080E82CC8A488104084FA
:10FAE000E42400C4EC440000000000008080208872
:10FAF000288020882088808020888020882CE8F03A
:10FB00000000000090909090101010108080808075
:10FB10007C8080801090B098408080440040646475
:10FB2000001800401C307800300C7C182800003091
:10FB300054181804400464186404282830400C1831
:10FB40007C4064606460606464180C78606468641D
:10FB5000607C780418643C7C3C1830600C18000011
:10FB6000002064606440306464180C50187C646445
:10FB70006C6C602430646464182C181818180C0C11
:10FB800080842088C4C444C420646430286C6C80A1
:10FB9000C0A08884000000008080808080807CEC91
:10FBA00018008044408440848080301880FC801895
:10FBB00000448040844444440000C004280024449D
:10FBC0001090282818302828000000000000244049
:10FBD000BCD0A41084404084E82CC8A44C8480800D
:10FBE000482400C4EC44000000000000808020880D
:10FBF000288020882088808020888020882CE82801
:10FC00000000000090909090101010108080808074
:10FC1000FC8080801090808084C4A8440000643CF4
:10FC20000000003C44686C00181818181800286080
:10FC3000641830640C646430640C281818001800D0
:10FC40007C6464646460606464186C6C60646464A4
:10FC500060686C6418643C7C641860600018000084
:10FC6000006464646460302064180C781864646410
:10FC7000482460043C683C7C3C0830181818041880
:10FC800044882088C4C4808064646818186C6C80C0
:10FC9000C0A0888400000080808080808080FCB4C8
:10FCA000400080804084208880843018DC80284098
:10FCB00000446040844444280000C0046C0024C414
:10FCC0001090440018306C0000000000000018186C
:10FCD000BCB0808084402088E44CC4C44C848080C4
:10FCE000282400C4EC440000000000008000282804
:10FCF000280028280000280028282820882CE83000
:10FD00000000000090909090101010108080808073
:10FD10007C4480441450808044EC442800004458C3
:10FD20000018003C18082C000C300000300028009F
:10FD3000242440240C242430242800300C003018C3
:10FD4000246444244440602464242864406464247B
:10FD5000602C64241824182464184048004800408B
:10FD6000002044242424300464246C6C246464241F
:10FD7000600C6044182C183C6404400C18300400DB
:10FD8000449040848080442820242C0000A8448093
:10FD9000C0A08884000080808080808040847C585F
:10FDA000240080288080208890A0600CDCFC44180F
:10FDB00000446040844444EC0000C0046C00240013
:10FDC00008A044000C606C00000000000000104817
:10FDD000BCB0808080801090D094C0048C8040841F
:10FDE000284000C4C444000000000000800028280F
:10FDF000280028280000280028282820882CE830FF
:10FE00000000000090909090101010108080808072
:10FE1000FC4480441450A8A84080440000006000C6
:10FE200000000000000000000000000000000000D2
:10FE300000000000000000000000000000000000C2
:10FE400000000000000000000000000000000000B2
:10FE500000000000000000000000000000000000A2
:10FE60000000000000000024000028000000000046
:10FE700060080000000000000024000000000000F6
:10FE800028A08080000000000000000000A844803E
:10FE9000C0A0888400808080808080804084FCECCA
:10FEA0001800444480801090A4A0C004DC806C3C06
:10FEB00000446000004400800080C004C4002400AE
:10FEC00008A080000C60C4000000000000000000DA
:10FED000A4B08080844008A0C8A480808C800000EA
:10FEE000444000808000000000000000000028283E
:10FEF000280028280000280028282824482CE8006A
:10FF00000000000090909090101010108080808071
:10FF10007C2880281450109080EC28000000C0003D
:10FF200000000000000000000000000000000000D1
:10FF300000000000000000000000000000000000C1
:10FF400000000000000000000000000000000000B1
:10FF500000000000000000000000000000000000A1
:10FF60000000000000000000000000000000000091
:10FF70000000000000000000000000000000000081
:10FF800028C0808000000000000000000000008009
:10FF9000C0A08884808080808080808020887C5879
:10FFA00000004480808008A004C0C0048CFCA858D5
:10FFB00000006000004400280080C004C40000006D
:10FFC00004C0800004C0C400000000000000000065
:10FFD0008080000084400000C8A400004824000085
:10FFE0000000000000000000000000008000282841
:10FFF000280028280000280028282828282CE80085
:00000001FF
